:100000000C9473000C949B000C949B000C949B002C
:100010000C949B000C94EB170C949B000C949B008D
:100020000C949B000C949B000C949B000C949B00E4
:100030000C949B000C949B000C949B000C949B00D4
:100040000C9419050C949B000C9401040C94DB0394
:100050000C949B000C949B000C949B000C949B00B4
:100060000C94B6050C949B004D0C4F0C510C530C8A
:10007000550C570C590C5B0C8D0C900C930C8A0C86
:10008000960C990CAA0CAA0C000000002400270072
:100090002A0000000000250028002B0000000000BE
:1000A00023002600290004040404040404040202BA
:1000B00002020202030303030303010204081020E7
:1000C00040800102040810200102040810200000F2
:1000D0000008000201000003040700000000000007
:1000E00000002629722A11241FBECFEFD8E0DEBF00
:1000F000CDBF26E0A4EEB3E001C01D92A136B20749
:10010000E1F713E0A0E0B1E0E8E8F4E602C0059012
:100110000D92A43EB107D9F710E0C2E7D0E004C0C9
:100120002197FE010E94772EC137D107C9F70E949F
:10013000D41A0C9437320C9400000895CF92DF92B9
:10014000EF92FF920F931F93CF93DF936C017A018D
:100150008B01C0E0D0E0CE15DF0589F0D8016D91AC
:100160008D01D601ED91FC910190F081E02DC60149
:100170000995892B11F47E0102C02196ECCFC701AD
:10018000DF91CF911F910F91FF90EF90DF90CF9073
:100190000895FC01538D448D252F30E0842F90E08D
:1001A000821B930B541710F0CF9608950197089572
:1001B000FC01918D828D981761F0828DDF01A80F6F
:1001C000B11D5D968C91928D9F5F9F73928F90E091
:1001D00008958FEF9FEF0895FC01918D828D981700
:1001E00031F0828DE80FF11D858D90E008958FEF3D
:1001F0009FEF0895FC01918D228D892F90E0805C06
:100200009F4F821B91098F739927089583ED94E086
:100210000E94FA0021E0892B09F420E0822F089542
:10022000FC01848DDF01A80FB11DA35ABF4F2C9193
:10023000848D90E001968F739927848FA689B78962
:100240002C93A089B1898C9180648C93938D848D3B
:10025000981306C00288F389E02D80818F7D80830A
:100260000895EF92FF920F931F93CF93DF93EC01CA
:1002700081E0888F9B8D8C8D981305C0E889F98962
:10028000808185FD24C0F62E0B8D10E00F5F1F4F7F
:100290000F731127E02E8C8DE8120CC00FB607FCEF
:1002A000FACFE889F989808185FFF5CFCE010E94D8
:1002B0001001F1CF8B8DFE01E80FF11DE35AFF4FC6
:1002C000F0820B8FEA89FB898081806207C0EE890A
:1002D000FF896083E889F98980818064808381E077
:1002E00090E0DF91CF911F910F91FF90EF900895D3
:1002F000CF93DF93EC01888D8823C9F0EA89FB89CD
:10030000808185FD05C0A889B9898C9186FD0FC0C3
:100310000FB607FCF5CF808185FFF2CFA889B98998
:100320008C9185FFEDCFCE010E941001E7CFDF91C8
:10033000CF91089580E090E0892B29F00E9406017A
:1003400081110C9400000895833081F028F48130ED
:1003500099F08230A1F008958730A9F08830B9F083
:100360008430D1F4809180008F7D03C08091800023
:100370008F7780938000089584B58F7702C084B50D
:100380008F7D84BD08958091B0008F7703C08091E8
:10039000B0008F7D8093B00008953FB7F8948091AE
:1003A000620490916304A0916404B091650426B541
:1003B000A89B05C02F3F19F00196A11DB11D3FBF9D
:1003C000BA2FA92F982F8827820F911DA11DB11D2B
:1003D000BC01CD0142E0660F771F881F991F4A9527
:1003E000D1F7089585ED8093BC008091BC0084FD19
:1003F000FCCF1092AE0408950895E09167048091B7
:100400006604E81730F4F0E0E859FB4F808190E093
:1004100008958FEF9FEF089590916704809166048F
:10042000981750F4E92FF0E0E859FB4F208130E0B5
:100430009F5F9093670402C02FEF3FEFC9010895BB
:100440008091660490E020916704821B91090895D1
:100450000E9419320F931F93CF93DF93EC01888191
:100460009981009729F02A813B812617370788F464
:100470008B016F5F7F4F0E944F31009761F099832E
:1004800088831B830A832C813D81232B11F4FC017B
:10049000108281E001C080E0DF91CF911F910F9128
:1004A0000895FC0180819181009711F00C94C62A77
:1004B00060E070E0CB010895FC0124813581232B9D
:1004C00031F421E061157105A1F0FB0108C0FC01C8
:1004D000808191816115710531F421E0FC018081F9
:1004E000882339F005C00E94273221E0892B09F0CA
:1004F00020E0822F0895EF92FF920F931F93CF93E6
:10050000DF93FC01248135816115710511F480E0D0
:1005100019C041155105A9F07B01EC018A01020FB8
:10052000131FB8010E942A02882389F32881398188
:100530008C819D81B701820F931F0E9430321D83F1
:100540000C8381E0DF91CF911F910F91FF90EF908D
:1005500008950F931F93CF93DF938C01EB01FC0160
:10056000808191810097B1F0688179816115710571
:1005700079F0428153812C813D814217530740F02D
:100580000E9430328C819D81F8019583848313C051
:100590000E94B73088819981F801918380838A8194
:1005A0009B81938382838C819D819583848319822F
:1005B00018821B821A821D821C82DF91CF911F91AB
:1005C0000F910895CF93DF93EC0188819981009773
:1005D00011F00E94B730198218821D821C821B8282
:1005E0001A82DF91CF910895CF93DF93EC01FB0145
:1005F00044815581608171810E947B02811103C019
:10060000CE010E94E202CE01DF91CF910895EF92D8
:10061000FF920F931F93CF93DF93EC017B018A012D
:10062000BA010E942A02811104C0CE010E94E20296
:1006300007C01D830C83B701888199810E943032E5
:10064000CE01DF91CF911F910F91FF90EF90089510
:10065000CF93DF93EC016115710559F0FB01019017
:100660000020E9F73197AF01461B570B0E940703A3
:1006700002C00E94E202CE01DF91CF910895CF9394
:10068000DF93EC01FB018617970761F060817181B0
:100690006115710529F0448155810E94070302C04C
:1006A0000E94E202CE01DF91CF910895FC0180818A
:1006B00091810C94B730FC01118210821382128256
:1006C000158214826115710551F0FB010190002023
:1006D000E9F73197AF01461B570B0C9407030895B8
:1006E000BF92CF92DF92EF92FF920F931F93CF931F
:1006F000DF937C016B018A01E9012417350720F49F
:10070000812F8901C42FD82F6BEA72E0C7010E94A4
:100710005B03D60114968D919C91159708171907C4
:10072000D0F48C179D0708F4EC01D601ED91FC91F3
:100730001197EC0FFD1FB08010824D915C91BA01B2
:10074000600F711FC7010E942803D601ED91FC9133
:10075000EC0FFD1FB082C701DF91CF911F910F9168
:10076000FF90EF90DF90CF90BF900895DC01ED9166
:10077000FC91DB0114964D915C9115976D917C91E4
:100780000280F381E02D09946115710579F0FB0178
:1007900001900020E9F73197AF01461B570BDC01B0
:1007A000ED91FC910280F381E02D099480E090E0CE
:1007B00008950C94C4031F920F920FB60F92112448
:1007C0002F933F934F935F936F937F938F939F9359
:1007D000AF93BF93EF93FF9383ED94E00E941001DA
:1007E000FF91EF91BF91AF919F918F917F916F9109
:1007F0005F914F913F912F910F900FBE0F901F90DF
:1008000018951F920F920FB60F9211242F938F936A
:100810009F93EF93FF93E091E304F091E4048081D0
:10082000E091E904F091EA0482FD12C09081809188
:10083000EC048F5F8F732091ED04821751F0E091EB
:10084000EC04F0E0ED52FB4F958F8093EC0401C077
:100850008081FF91EF919F918F912F910F900FBE0B
:100860000F901F901895CF93DF93282F30E0F90158
:10087000E253FF4F8491F901E654FF4FD491F901FF
:10088000EA55FF4FC491CC2391F081110E94A4013D
:10089000EC2FF0E0EE0FFF1FE456FF4FA591B4914F
:1008A000EC91ED2381E090E021F480E002C080E053
:1008B00090E0DF91CF9108951F93CF93DF93282F7E
:1008C00030E0F901E253FF4F8491F901E654FF4F04
:1008D000D491F901EA55FF4FC491CC23C9F0162FEA
:1008E00081110E94A401EC2FF0E0EE0FFF1FEE56E5
:1008F000FF4FA591B4918FB7F894111105C09C9149
:10090000ED2FE095E92302C0EC91ED2BEC938FBF26
:10091000DF91CF911F910895CF93DF9390E0FC0179
:10092000E654FF4F2491FC01EA55FF4F8491882340
:1009300061F190E0880F991FFC01E857FF4FC591C6
:10094000D491FC01EE56FF4FA591B491611109C0FD
:100950009FB7F8948881209582238883EC912E2379
:100960000BC0623061F49FB7F8943881822F809574
:1009700083238883EC912E2B2C939FBF06C08FB7C7
:10098000F894E8812E2B28838FBFDF91CF910895B3
:100990008E3008F08E508770806480937C00809148
:1009A0007A00806480937A0080917A0086FDFCCF83
:1009B000809178002091790090E0922B08958F9299
:1009C0009F92AF92BF92CF92DF92EF92FF926B0114
:1009D0007C010E94CD014B015C01C114D104E104F2
:1009E000F104F1F00E94CD01DC01CB0188199909D5
:1009F000AA09BB09883E9340A105B10570F321E027
:100A0000C21AD108E108F10888EE880E83E0981E2A
:100A1000A11CB11CC114D104E104F10419F7DDCF0C
:100A2000FF90EF90DF90CF90BF90AF909F908F900E
:100A300008951F920F920FB60F9211242F933F9398
:100A40008F939F93AF93BF938091E4039091E503BD
:100A5000A091E603B091E7033091610423E0230FF6
:100A60002D3720F40196A11DB11D05C026E8230FE6
:100A70000296A11DB11D209361048093E40390931D
:100A8000E503A093E603B093E7038091620490919D
:100A90006304A0916404B09165040196A11DB11D89
:100AA0008093620490936304A0936404B0936504FC
:100AB000BF91AF919F918F913F912F910F900FBE5A
:100AC0000F901F901895FC01248131E03093AF0402
:100AD0002093D1041092B0041092D2048385682B25
:100AE00080E795E00E945C130C94AB0A0F931F9370
:100AF000CF938C01C62F0E9463056C2F6460C801E0
:100B00000E9463056C2F6B7FC8010E94630583EC14
:100B100090E00197F1F7CF911F910F910895FF9207
:100B20000F931F93CF93DF931F92CDB7DEB78C0146
:100B3000F62E962F907F692F642BC80149830E945F
:100B4000760580E1F89EB00111244981642BC8012B
:100B50000F90DF91CF911F910F91FF900C9476052C
:100B600041E00E948F0581E090E008951F920F926E
:100B70000FB60F9211242F933F934F935F936F9370
:100B80007F938F939F93AF93BF93EF93FF93809146
:100B9000B900887F803609F49CC068F5883209F472
:100BA0005BC090F4803109F454C038F4882309F410
:100BB000F6C0883009F44DC0F6C0883109F44CC045
:100BC000803209F45DC0EFC0803409F468C048F495
:100BD000803309F455C0883309F0E5C08093AC0434
:100BE000D8C0803509F44FC0883509F45DC0883419
:100BF00009F0D9C0D6C0883909F4C7C0A8F488372D
:100C000009F467C038F4883609F463C0803709F402
:100C100060C0C9C0883809F4B8C0803909F45FC021
:100C2000803809F0C0C05BC0803B09F486C038F44E
:100C3000803A09F466C0883A09F47FC0B4C0803CA9
:100C400009F4A7C0883C09F4A4C0883B09F48AC011
:100C5000AAC08091890410C09091AB048091AA042D
:100C6000981770F5E091AB0481E08E0F8093AB0490
:100C7000F0E0E657FB4F80818093BB0085EC86C097
:100C80008093AC048EC0E091AB0481E08E0F809322
:100C9000AB048091BB00F0E0E657FB4F808390915E
:100CA000AB048091AA046EC0E091AB0481E08E0F8A
:100CB0008093AB048091BB00F0E0E657FB4F80834C
:100CC0008091AD0481116DC081E08093880484EA35
:100CD00061C083E08093AE0410926004CFCF809116
:100CE0006004803208F051C0E091600481E08E0F12
:100CF000809360048091BB00F0E0E05CFB4F808358
:100D0000BDCF85EC8093BC001092AE04809160044E
:100D1000803230F4E0916004F0E0E05CFB4F108240
:100D20006091600470E0E0913E04F0913F0480E443
:100D300094E009951092600436C084E08093AE047C
:100D400010923D0410923C04E0913A04F0913B046F
:100D5000099580913C04811105C081E080933C0499
:100D600010921A04E0913D0481E08E0F80933D04BF
:100D7000F0E0E65EFB4F80818093BB0090913D04E4
:100D800080913C04981708F479CF85E88093BC00E3
:100D90000AC085EC8093BC001092AE0404C010928F
:100DA000AC040E94F201FF91EF91BF91AF919F912E
:100DB0008F917F916F915F914F913F912F910F9004
:100DC0000FBE0F901F90189540913C04262F30E0E5
:100DD000240F311D21323105DCF42091AE04243082
:100DE000C9F4FC0180E090E0861758F430913C048F
:100DF0002191DC01A65EBB4FA30FB11D2C93019680
:100E0000F3CF80913C04680F60933C0480E0089528
:100E100081E0089582E00895CF92DF92EF92FF92F1
:100E20000F931F93CF93DF937C01262F972F8A0177
:100E30008091AF04882391F0C62FD72F6E01C40E86
:100E4000D51ECC15DD0571F06991D701ED91FC91AE
:100E50000190F081E02DC7010995F3CF642F822F17
:100E60000E94E406C801DF91CF911F910F91FF907E
:100E7000EF90DF90CF9008951092AE0481E08093C0
:100E8000AD041092880461E082E10E945C0461E09C
:100E900083E10E945C04E9EBF0E080818E7F808337
:100EA00080818D7F808388E48093B80085E480937F
:100EB000BC0008952F923F924F925F926F927F9263
:100EC0008F929F92AF92BF92CF92DF92EF92FF925A
:100ED0000F931F93CF93DF93CDB7DEB76A970FB60B
:100EE000F894DEBF0FBECDBF322E232E4D875E8716
:100EF0003B012C01A982B98ACA8ADB8AEC8AFD8A65
:100F00000E8B1F8B988A8F86211500EA30070CEA1A
:100F1000400709EB500703E0600771058105910563
:100F200011F008F046C02F3F10EE310715EF4107D2
:100F300015E05107610571058105910561F058F0D3
:100F40002F3F354D41415E47634071058105910555
:100F500009F0D8F50BC0312CB1EE2B2EF5EFFD8743
:100F600005E00E87612C712C412C512C2981398987
:100F70004A895B896C897D898E899F89A0E00E945E
:100F8000023009F0AEC0A32CB22CCD84DE847301F4
:100F9000820120E034E04BE654EF64E170E080E051
:100FA00090E00E94432F29873A874B875C87912CDA
:100FB00024C0312CF0EA2F2E1CEA1D8729EB2E8746
:100FC000A3E06A2E712C412C512C298139894A8940
:100FD0005B896C897D898E899F89A0E00E9402309F
:100FE00009F025C19924939414E0E12EF12C00E03E
:100FF00010E0E986FA860B871C87E984FA840B8562
:101000001C85A801970160E070E0CB01A32CB22CF5
:10101000CD84DE847301820129833A834B835C8310
:101020006D837E838F83988760E070E080E090E03E
:101030000E947D2E2983398B4A8B5B8B6C8B7D8B39
:101040008E8B9F8BFF24F3949F1409F4F3C010E060
:10105000812C912C54018394C12CD12C760101C098
:1010600011E007E0CC0CDD1CEE1CFF1C0A95D1F74B
:10107000C701B601A50194010E94362E89859A8583
:10108000AB85BC8567E0880F991FAA1FBB1F6A95B7
:10109000D1F79250A109B109820F931FA41FB51F68
:1010A000EF85F88980839183A283B383C501B4015E
:1010B0000E94122EC61AD70AE80AF90AC482D582FB
:1010C000E682F78280869186A286B3861111E5C0FA
:1010D000298139894A895B896C897D898E899F89B3
:1010E000E2C01A8EA32CB22CCD84DE84730182015F
:1010F000298139894A895B896C897D898E899F8993
:101100000E94432F29873A874B875C8789859A8578
:10111000AB85BC850697A105B10520F4F6E0AF2E9E
:10112000B12C0FC0E984FA840B851C8529E0E216F6
:1011300027E0F20601051105D0F078E0A72EE7E0E0
:10114000BE2EC12CD12CE12CF12C00E010E0298125
:1011500039894A895B896C897D898E899F890E943A
:10116000432F322E232E4D875E873B012C01A32C6B
:10117000B22CCD84DE8473018201298139894A89A8
:101180005B896C897D898E899F890E94412F4901E5
:10119000B42FA52FF62FE72F888F998F05E00E9497
:1011A000B02F5401CB2EDA2EEF2EFE2E088D198D86
:1011B0000E94F02F05E00E94B02F088D0E94E72FBB
:1011C00005E00E94B02F088D0E94F02F288F398FE4
:1011D0004A01B62FA72FF82FE92F6B2F7A2F8F2FC9
:1011E0009E2F05E00E94B02F59016A017B018C01FE
:1011F000288D398DA4016B2F7A2F8F2F9E2F0E945F
:10120000E72FA32CB22CCD84DE84730182010E94CF
:10121000432FC22ED32EE42EF52EC114D104E104A7
:10122000F104F9F4812C912C5401839420C081E0C5
:101230008A8F58CFAF85B8891D921D921D921C923E
:101240001397FD011482158216821782C12CD12CAE
:101250007601C3941896CD92DD92ED92FC921B9785
:1012600022C088248A94982C8FE0A82EB12CFA8D65
:10127000F13009F0F5CEEF85F889108211821282E3
:101280001382148215821682178281E090E0A0E01A
:10129000B0E080879187A287B387232D322D4D85BB
:1012A0005E85B301C2016A960FB6F894DEBF0FBE29
:1012B000CDBFDF91CF911F910F91FF90EF90DF9005
:1012C000CF90BF90AF909F908F907F906F905F90E6
:1012D0004F903F902F900895DF92EF92FF920F93DF
:1012E0001F93CF93DF93FC01E080F1800281138193
:1012F000D481C581B681D7809701A8016D2F7C2F3D
:101300008B2F9D2D35534C4051096109710981097D
:1013100091092F3F34434C4051056105710581050A
:10132000910509F098F49701A8016D2F7C2F8B2F60
:101330009D2D07E00E94B02F208331834283538389
:10134000648375838683978387E0FDC09701A80136
:101350006D2F7C2F8B2F9D2D3A56484151096109E5
:101360007109810991092F3F3946484151056105AD
:1013700071058105910509F098F49701A8016D2F79
:101380007C2F8B2F9D2D06E00E94B02F2083318370
:1013900042835383648375838683978386E0D3C0B7
:1013A0009701A8016D2F7C2F8B2F9D2D345D40431D
:1013B000510961097109810991092F3F334D40435A
:1013C0005105610571058105910509F098F49701B2
:1013D000A8016D2F7C2F8B2F9D2D05E00E94B02F33
:1013E0002083318342835383648375838683978309
:1013F00085E0A9C09701A8016D2F7C2F8B2F9D2D13
:10140000385A4146510961097109810991092F3FF3
:10141000374A41465105610571058105910509F07D
:1014200098F49701A8016D2F7C2F8B2F9D2D04E040
:101430000E94B02F2083318342835383648375835A
:101440008683978384E07FC09701A8016D2F7C2F4E
:101450008B2F9D2D3055434C51096109710981092C
:1014600091092F3F3F44434C5105610571058105AA
:10147000910509F098F49701A8016D2F7C2F8B2F0F
:101480009D2D03E00E94B02F20833183428353833C
:10149000648375838683978383E055C09701A80191
:1014A0006D2F7C2F8B2F9D2D305A4648514061095E
:1014B0007109810991092F3F3F4946485140610513
:1014C00071058105910509F098F49701A8016D2F28
:1014D0007C2F8B2F9D2D02E00E94B02F2083318323
:1014E00042835383648375838683978382E02BC012
:1014F0009701A8016D2F7C2F8B2F9D2D30544D40CF
:10150000534061097109810991092F3F3F434D40C3
:101510005340610571058105910509F098F4970123
:10152000A8016D2F7C2F8B2F9D2D01E00E94B02FE5
:1015300020833183428353836483758386839783B7
:1015400081E001C080E0DF91CF911F910F91FF906A
:10155000EF90DF9008952091D2049091D104213230
:1015600008F04AC08091AE048111FCCF32E0309384
:10157000AE0431E03093AD043FEF3093AC041092F1
:10158000AB042093AA04A1EBB4E04AE854E0FA01CA
:101590003E2F341B321718F43D913193F9CF10923E
:1015A000890420918904990F922B9093890490913A
:1015B0008804913061F4109288049091890490938A
:1015C000BB009091BC0093FDF8CF95EC01C095EE67
:1015D0009093BC009091AE049230E1F39091AC04F2
:1015E0009F3F79F08091AC04803241F08091AC044F
:1015F000803331F084E005C081E003C082E001C0A7
:1016000083E01092B0041092D2041092AF040895B7
:10161000EF92FF920F931F93CF93DF931F92CDB75B
:10162000DEB7162F91E09093AF0490E69093D1042B
:101630001092B0041092D204682F80E795E079836D
:101640000E945C13E12E7981F72E8701085F1F4FFE
:10165000F70161917F0180E795E00E945C13E0163D
:10166000F106B1F70F90DF91CF911F910F91FF908D
:10167000EF900C94AB0AEF92FF920F931F93CF93CE
:10168000DF931F92CDB7DEB7162F877028E0829FB9
:10169000C0011124682F606440E08FE396E07983F5
:1016A0000E948F05E12E7981F72E8701085F1F4F79
:1016B000F70161917F018FE396E00E94B005E0168B
:1016C000F106B1F70F90DF91CF911F910F91FF902D
:1016D000EF900895CF93C62F91E09093AF0490E6DA
:1016E0009093D1041092B0041092D204682F80E736
:1016F00095E00E945C136C2F80E795E00E945C13DC
:10170000CF910C94AB0ACF93DF9391E09093AF0409
:1017100090E69093D1041092B0041092D204682FF6
:1017200080E795E00E945C130E94AB0A8091AE04B2
:101730008111FCCF91E09093AE041092AD048FEF35
:101740008093AC041092AB041092AA049093890485
:1017500090918904906C90938904809188048130E1
:1017600061F410928804809189048093BB00809179
:10177000BC0083FDF8CF85EC01C085EE8093BC00F2
:101780008091AE048130E1F38091AB04811103C0FC
:10179000C091AB0401C0C1E0AAE8B4E028E634E09F
:1017A000F9018E2F821B8C1718F48D918193F9CF3C
:1017B00010926704C093660480916704C81731F0E3
:1017C00080E795E00E940C02D82FF6CF8D2FDF9195
:1017D000CF9108952F923F924F925F926F927F9296
:1017E0008F929F92AF92BF92CF92DF92EF92FF9231
:1017F0000F931F93CF93DF93CDB7DEB72E970FB61E
:10180000F894DEBF0FBECDBF982E792E49875A8738
:101810006B877C876BA05C2C2D2C3E2D402E312EAF
:10182000C984DA84EB84FC8484E190E02E873D87D0
:101830000E9422308C01FC01D082C182892D880F48
:10184000880F880F845D0E94830B8C7F3D85932FCA
:101850009370892BF801828323825482D701C601B9
:101860006CE0B695A795979587956A95D1F7982FCF
:10187000907F2E85822F8F70C82EC90EC58236822A
:101880004782E92CF72CF8E0EF16F104B8F4F701E1
:10189000EC5CFF4FB8010C94772E8AE20DC082E316
:1018A0000BC08AE309C082E407C08AE405C082E570
:1018B00003C08AE501C08BE50E94080B80E1980E09
:1018C000892D0E94830B91E0682FA91202C06064E9
:1018D00001C06F7B892D0E946A0BE1E0EE16F104D6
:1018E00051F0F2E0EF16F10449F0E114F10449F48B
:1018F000A092320612C0A092330612C0A092340603
:1019000012C088E0E816F104B0F4F701E45CFF4F80
:101910000C94772E54E4B52E0EC04CE2B42E0BC0BE
:1019200034E3B32E08C02CE3B22E05C09CE4B92EDC
:1019300002C084E5B82E8B2D0E94830B8378611042
:101940008C6090E1899E40011124682F68298B2DBD
:101950000E946A0BC8012E960FB6F894DEBF0FBE28
:10196000CDBFDF91CF911F910F91FF90EF90DF904E
:10197000CF90BF90AF909F908F907F906F905F902F
:101980004F903F902F900C94B7300F931F93CF93AD
:101990008B01C0E1C80F8C2F0E94830B011511052C
:1019A00011F48F7D04C00130110509F48062682FA5
:1019B0008C2FCF911F910F910C946A0B2F923F9215
:1019C0004F925F926F927F928F929F92AF92BF924F
:1019D000CF92DF92EF92FF920F931F93CF93DF93FB
:1019E000CDB7DEB763970FB6F894DEBF0FBECDBF9D
:1019F000322E3A874B875C876D87272E2C011F87F5
:101A00000E8760913B0670913C0680913D06909157
:101A10003E0624E630E040E050E00E94E52E2A8BAE
:101A20003B8B4D835E83762E672E888B998B8091BE
:101A3000350690913606A0913706B09138066C01B4
:101A40007D01FF0CCC08DC2C76019C01AD016C2DD6
:101A50007C2D8C2D9C2D0FE10E94B02FA12CEAEC47
:101A6000BE2EFAE9CF2EABE3DA2EE12CF12C00E00A
:101A700010E00E94122FAA88BB88CD80DE80E72C60
:101A8000F62C088919890E947D2E0FE10E94CB2F28
:101A900049015A01D501C401BB0F880B982FDC0105
:101AA00089839A83AB83BC839401A5016981762FD6
:101AB000862F962FAA88BB88CD80DE80E72CF62C57
:101AC00008890E94E72F39014A01698B788B898345
:101AD0009D83232D3A854B855C856D85722DC201D2
:101AE0002F3FA7E53A07A7E44A07A8EF5A07ADE05A
:101AF0006A07710581059105A9F0A0F02115344010
:101B00004B46544F6441710581059105B9F0B0F021
:101B1000312CA4E0AA87BBE6BB87E4EFEC87F4E1B5
:101B2000FD8709C0312CE8E5EA87F7E4FB8788EFF9
:101B30008C879DE09D87212C412C512C5301640101
:101B4000E988F88809811D81232D3A854B855C85BC
:101B50006D85722DC2010E94432F2E833F834887DB
:101B600059878E819F81A885B9850F97A105B105F9
:101B700058F49301A401B701C80104E00E94B02FFA
:101B800009810E94F02F28C08E819F81A885B98588
:101B90008B359105A105B10530F19301A401698947
:101BA000788989819D8102E00E94B02F53016401F0
:101BB000E988F88809811D810E94F02F59016A0186
:101BC0007B01E82F192F04E00E94B02F0E2F0E94F6
:101BD000F02F01E00E94B02F322E3A874B875C87AE
:101BE0006D87272E2C0153016401E988F88809814B
:101BF0001D81232D3A854B855C856D85722DC20133
:101C00000E94412F2901B42FA52FF62FE72F382E40
:101C1000292E05E00E94B02F5201CB2EDA2EEF2E96
:101C2000FE2E032D122D0E94F02F05E00E94B02FF2
:101C3000032D0E94E72F05E00E94B02F032D0E9484
:101C4000F02F19012A01B62FA72FF82FE92F05E051
:101C50000E94B02F59016A017B018C019101A20100
:101C60006B2F7A2F8F2F9E2F0E94E72F5301640135
:101C7000E988F88809811D810E94432F69017A0152
:101C8000C114D104E104F10429F4812C912C5401F4
:101C9000839406C088248A94982C3FE0A32EB12C0C
:101CA00087E0CC0CDD1CEE1CFF1C8A95D1F7C70128
:101CB000B601A50194010E94362E4E805F80688493
:101CC000798497E0440C551C661C771C9A95D1F7D3
:101CD00092E0591A61087108420E531E641E751E67
:101CE000C501B4010E94122EC61AD70AE80AF90AE1
:101CF00084E190E00E9422308C01DC019C921196DC
:101D00008C921197862D837012968C93129713964E
:101D10005C92139714964C92D501C4012CE0B695B1
:101D2000A795979587952A95D1F7982F907F8E2D17
:101D30008F70882E890EF8018582D682C7828E85A3
:101D40009F85892B19F4B8018AE106C0AE85BF854D
:101D5000119721F4B80182E20E94080BC801639632
:101D60000FB6F894DEBF0FBECDBFDF91CF911F91AC
:101D70000F91FF90EF90DF90CF90BF90AF909F902A
:101D80008F907F906F905F904F903F902F900C942A
:101D9000B7302F923F924F925F926F927F928F92C5
:101DA0009F92AF92BF92CF92DF92EF92FF920F93EA
:101DB0001F93CF93DF93CDB7DEB7AB970FB6F894F1
:101DC000DEBF0FBECDBF298F3A8F4B8F5C8F6D8FDB
:101DD0007E8F8F8F98A37A2CB9A2CAA2DBA23E2C49
:101DE0004F2C602E212E9AA689A62A2D3B2DA601C6
:101DF0006E2D7F2D802F912FA0E00E94023091F058
:101E000038554744584F6D40710981099109211592
:101E10003C4A43425C4F664071058105910511F0D3
:101E200008F028C4298D3A8D4B8D5C8D6D8D7E8D8B
:101E30008F8D98A12F3F34434C40510561057105AA
:101E40008105910509F050F4198E85E38A8F8CE0A5
:101E50008B8F1C8E1D8E1E8E1F8E18A2298D3A8D83
:101E60004B8D5C8D6D8D7E8D8F8D98A12115304AA7
:101E70004C4A594B634071058105910569F060F04A
:101E8000198E80EA8A8F8CEA8B8F89EB8C8F83E0A6
:101E90008D8F1E8E1F8E18A2CE0149960E946C094E
:101EA0008BA7272D39A14AA15BA1632D742D862D07
:101EB000922DA0E0B98DFA8DEB8D0E94023009F4CD
:101EC00083C0AC8D8D8D5E8C9F8D9EA318A118A7AD
:101ED0002B2F3F2F4E2F5A2F682F752D892F912F83
:101EE0002F3F15ED310711E141071EE7510713E0C0
:101EF000610771058105910511F008F065C0CE01FB
:101F00000D964C01A72CB9A0CAA0DBA0E32CF42CA1
:101F1000062D122D8EA198A50E945A0789A59AA573
:101F200081309105F9F082309105A9F1892B09F0F2
:101F30007AC3898D80931A068A8D80931B068B8DB8
:101F400080931C068C8D80931D068D8D80931E06BC
:101F50008E8D80931F068F8D8093200688A180939D
:101F6000210661C3898D809322068A8D8093230682
:101F70008B8D809324068C8D809325068D8D809388
:101F800026068E8D809327068F8D8093280688A144
:101F90008093290648C3898D80932A068A8D809371
:101FA0002B068B8D80932C068C8D80932D068D8D2A
:101FB00080932E068E8D80932F068F8D8093300612
:101FC00088A1809331062FC39C8D1D8D1CA35E8C30
:101FD0008F8D8EA3A8A12B2F3F2F4E2F592F612F0E
:101FE000752D9A2F2F3F15ED310711E141071EE79F
:101FF000510713E06107710581059105D9F0D0F013
:10200000CE010D964C01A12CB12CC12CD12CE12C70
:10201000F12C00E010E08EA19A2F0E945A07722E38
:1020200039A34AA35BA3362E472E682E292E91E0B2
:102030009FA301C01FA289A59AA58130910509F42B
:102040005AC08230910509F4A0C1892B09F012C34E
:10205000298D3A8D4B8D5C8D6D8D7E8DCE010D96CB
:102060004C01A12CB12CC12CD12CE12CF12C00E085
:1020700010E08F8D98A10E945A07722E39A34AA3AF
:102080005BA3362E472E682E292E60E070E080E09C
:1020900090E00E94C50C70920A0699A190930B06DD
:1020A000EAA1E0930C061BA110930D0630920E06D8
:1020B00040920F066092100620921106898D80933F
:1020C0001A068A8D80931B068B8D80931C068C8D3F
:1020D00080931D068D8D80931E068E8D80931F0626
:1020E0008F8D8093200688A18093210655245394D8
:1020F0001DA21CA29AC280913A06E98DECA3EA8D3A
:10210000EEA3EB8DE8A75C8CBD8DAE8DFF8DE8A1B5
:10211000823009F075C02CA13EA148A5552D6B2F2A
:102120007A2F8F2F9E2F30584A41564061097109EE
:10213000810991092F37304E424758496240710555
:102140008105910569F160F1A0902A06B0902B06F7
:10215000C0902C06D0902D06E0902E06F0902F0611
:1021600000913006109131062CA13EA148A5552DB5
:102170006B2F7A2F8F2F9E2F0E94F92F89F01092AC
:102180002206109223061092240610922506109221
:1021900026061092270610922806109229066AC277
:1021A000709012068091130689A3909114069AA349
:1021B000109115061BA330901606409017066090EC
:1021C000180620901906CE010D964C01A72CB9A037
:1021D000CAA0D12EE32CF42C062D122D2CA13EA149
:1021E00048A5552D6B2F7A2F8F2F9E2F0E945A07AF
:1021F00061E070E081E090E00E94C50C512C38C095
:102200007092120699A1909313061AA110931406C6
:102210008BA18093150630921606409217066092A5
:10222000180620921906CE010D964C01A12CB12C56
:10223000C12CD12CE12CF12C00E010E02CA13EA10E
:1022400048A5552D6B2F7A2F8F2F9E2F0E945A074E
:10225000722E39A34AA35BA3362E472E682E292E51
:1022600061E070E081E090E00E94C50C5524539439
:10227000298D3A8D4B8D5C8D6D8D7E8D8F8D98A1C6
:1022800030584A41564061097109810991092F3737
:10229000304E42475849624071058105910509F069
:1022A00008F457C081E080933A0620912A063091C5
:1022B0002B0640912C0650912D0660912E067091B0
:1022C0002F068091300690913106A0E00E940230E6
:1022D00009F442C08AE296E00E946C098BA7A090A4
:1022E0001206B0901306C0901406D0901506E09028
:1022F0001606F09017060091180610911906209105
:102300002A0630912B0640912C0650912D066091A3
:102310002E0670912F06CE0101964C018091300659
:10232000909131060E945A071F928BA4A12CC9805C
:10233000DA80EB80FC800D811E812F8138854985F4
:102340005A856B857C8582E090E00E94EA0B0F90B5
:1023500003C088E080933A06898D809322068A8D97
:10236000809323068B8D809324068C8D8093250685
:102370008D8D809326068E8D809327068F8D80937A
:10238000280688A18093290649C190903A06E98DD4
:10239000ECA3EA8DEEA3EB8DE8A75C8CBD8DAE8D32
:1023A000FF8DE8A111E0911275C02CA13EA148A5B6
:1023B000552D6B2F7A2F8F2F9E2F30584A41564024
:1023C00061097109810991092F37304E42475849F7
:1023D000624071058105910569F160F1A0902A06BE
:1023E000B0902B06C0902C06D0902D06E0902E06C3
:1023F000F0902F0600913006109131062CA13EA1DD
:1024000048A5552D6B2F7A2F8F2F9E2F0E94F92FC5
:1024100089F010922A0610922B0610922C06109228
:102420002D0610922E0610922F0610923006109252
:10243000310624C1709012068091130689A39091F1
:1024400014069AA3109115061BA33090160640900F
:1024500017066090180620901906CE010D964C01C3
:10246000A72CB9A0CAA0D12EE32CF42C062D122D36
:102470002CA13EA148A5552D6B2F7A2F8F2F9E2F73
:102480000E945A0761E070E082E090E00E94C50C73
:10249000512C38C07092120699A1909313061AA17C
:1024A000109314068BA18093150630921606409265
:1024B00017066092180620921906CE010D964C015F
:1024C000A12CB12CC12CD12CE12CF12C00E010E07E
:1024D0002CA13EA148A5552D6B2F7A2F8F2F9E2F13
:1024E0000E945A07722E39A34AA35BA3362E472EA9
:1024F000682E292E61E070E082E090E00E94C50C19
:1025000055245394298D3A8D4B8D5C8D6D8D7E8D28
:102510008F8D98A130584A4156406109710981094F
:1025200091092F37304E4247584962407105810565
:10253000910509F008F457C082E080933A06209193
:102540002206309123064091240650912506609181
:102550002606709127068091280690912906A0E012
:102560000E94023009F442C082E296E00E946C09A7
:102570008BA7A0901206B0901306C0901406D090BE
:102580001506E0901606F0901706009118061091B7
:10259000190620912206309123064091240650917D
:1025A00025066091260670912706CE0101964C0102
:1025B00080912806909129060E945A071F928BA4A9
:1025C000A12CC980DA80EB80FC800D811E812F81D7
:1025D000388549855A856B857C8581E090E00E942D
:1025E000EA0B0F9003C088E080933A06898D8093B0
:1025F0002A068A8D80932B068B8D80932C068C8DDA
:1026000080932D068D8D80932E068E8D80932F06C0
:102610008F8D8093300688A18093310681E090E011
:102620009DA38CA302C01FA2512C9FA19F938BA49A
:10263000AFA0CD84DE84EF84F88809891A892B89BC
:102640003C894D895E896F89788D89A59AA50E94FC
:10265000EA0B0F90E1E05E1210C00CA11DA1272D26
:1026600039A14AA15BA1632D742D862D922D0E9464
:10267000DE0C03C09924939401C0912C892DAB9654
:102680000FB6F894DEBF0FBECDBFDF91CF911F9183
:102690000F91FF90EF90DF90CF90BF90AF909F9001
:1026A0008F907F906F905F904F903F902F90089504
:1026B000089580E090E00895CF93DF931F92CDB707
:1026C000DEB769832091AF042223D1F02091D20498
:1026D000203240F021E030E0FC013383228380E0AF
:1026E00090E015C08091B004E82FF0E0EF54FB4F6C
:1026F000998190838F5F8093B0048093D20405C04A
:1027000061E0CE0101960E94E40681E090E00F9026
:10271000DF91CF910895CF92DF92EF92FF920F93C6
:102720001F93CF93DF93EB017B0124E0E20EF11CBA
:102730008B016C01C61AD70AC601800F911F0E9437
:102740008C2CF80181938F01EE15FF05A9F7CE01BE
:10275000DF91CF911F910F91FF90EF90DF90CF907D
:102760000895AF92BF92CF92DF92EF92FF920F93B4
:102770001F93CF93DF931F92CDB7DEB75C017B0130
:102780008B016C0184E0C80ED11CF80161918F01AE
:10279000C50169830E948C2C6981681719F0C501F5
:1027A0000E94942CFFEFAF1ABF0AAC14BD0469F766
:1027B000C7010F90DF91CF911F910F91FF90EF9084
:1027C000DF90CF90BF90AF900895CF93DF93EC014F
:1027D00060E471E08AE090E00E948B13FC0180814C
:1027E0009181A281B3818093400190934101A09394
:1027F0004201B09343016CE371E084E190E00E94F8
:102800008B13FC0180819181A281B38180933C0173
:1028100090933D01A0933E01B0933F018091E90365
:102820009091EA03009769F58091ED03813009F4F6
:102830006CC0C130D10561F48091EE039091EF033B
:10284000A091F003B091F1030196A11DB11D10C03C
:10285000CF3FFFEFDF0709F058C08091EE03909162
:10286000EF03A091F003B091F1030197A109B10921
:102870008093EE039093EF03A093F003B093F103E2
:1028800044C0019709F041C0C130D105A9F440917D
:10289000400150914101609142017091430180914A
:1028A000440190914501A0914601B0914701840FE8
:1028B000951FA61FB71F18C0CF3F2FEFD20711F5E6
:1028C0008091400190914101A0914201B09143015A
:1028D000409144015091450160914601709147013A
:1028E000841B950BA60BB70B80934001909341017D
:1028F000A0934201B093430160E471E08AE090E06C
:102900000E94B11381E0809358068091E903909171
:10291000EA03029709F04AC0C130D10539F5809128
:102920003C0190913D01A0913E01B0913F01805F3B
:10293000984DAF4FBF4F8038E3EC9E07E9ECAE07F0
:10294000E1E0BE0724F080E893ECA9ECB1E08093CD
:102950003C0190933D01A0933E01B0933F016CE395
:1029600071E084E190E00E94B1131DC0CF3FFFEF02
:10297000DF07C9F480913C0190913D01A0913E0197
:10298000B0913F0180519742A109B109813026E3FE
:1029900092072EE6A20721E0B207CCF680E096E38C
:1029A000AEE6B1E0D4CF81E0809358068091E90390
:1029B0009091EA03039709F04AC0C130D10539F577
:1029C00080917C0590917D05A0917E05B0917F0559
:1029D000805C944BA34BBF4F8115E9EE9E07E4EA60
:1029E000AE07E5E3BE0724F080E099EEA4EAB5E384
:1029F00080937C0590937D05A0937E05B0937F0521
:102A00006CE775E08EE190E00E94B1131DC0CF3FEE
:102A1000FFEFDF07C9F480917C0590917D05A091BF
:102A20007E05B0917F0580549B44AC44B109813050
:102A300026E4920723ECA20723E2B207CCF680E05B
:102A400096E4A3ECB3E2D4CF81E080935806809162
:102A5000E9039091EA030497B1F58091ED03813089
:102A600091F1C130D10539F5809154018F5F8230E9
:102A700008F082E08093540180915401813029F460
:102A800080E091EEA0E0B0E006C0823061F480E02A
:102A900092ECA1E0B0E08093380190933901A093CB
:102AA0003A01B0933B0168E371E088E290E0DF9186
:102AB000CF910C94B113219631F48091540181503F
:102AC000C9F681E0D7CFDF91CF91089580E10E94D0
:102AD0003304892B61F48091EC03811108C080914B
:102AE000EB03811104C080915C06882329F080915A
:102AF0005B06813009F06EC081E08093E80381E1DC
:102B00000E943304892B59F48091590690915A06FA
:102B1000892B29F480915806882309F45EC081E14D
:102B20000E943304019739F48091590690915A0616
:102B3000019709F470C08091E9039091EA0301972D
:102B4000E9F480915C06811119C08091480190914F
:102B50004901A0914A01B0914B0180935206909394
:102B60005306A0935406B09355066EEC75E086EBC1
:102B700095E00E943F0381E080935C0685E00E941F
:102B80003304019739F48091500690915106892BB6
:102B900009F446C085E00E943304892B39F4809102
:102BA000500690915106019709F44FC080914E064E
:102BB00090914F06009731F481E08093EC0380936D
:102BC000EB030895019709F045C01092EC031092B1
:102BD000EB0308951092E80392CF81E090E02091FA
:102BE000560630915706232B11F080E090E0909329
:102BF00057068093560681E090E090935A068093A2
:102C000059068091E9039091EA0301969093EA03B3
:102C10008093E90384CF10925A06109259068BCF05
:102C200081E090E020914E0630914F06232B11F069
:102C300080E090E090934F0680934E0681E090E014
:102C40009093510680935006A5CF10925106109292
:102C50005006ACCF08958F929F92AF92BF92CF92C1
:102C6000DF92EF92FF920F931F93CF93DF93CDB735
:102C7000DEB7AE970FB6F894DEBF0FBECDBF809122
:102C8000E9039091EA03019709F067C060E080E0F2
:102C90000E94541A6BE573E08FE396E00E94D9031B
:102CA00061E080E00E94541A6CE673E08FE396E0E6
:102CB0000E94D903609140017091410180914201CD
:102CC000909143010E94841A80E20E94301980E2B0
:102CD0000E94301980E20E9430191092ED03109288
:102CE000E80310925B066CE472E083ED94E00E94CE
:102CF000D90364E773E083ED94E00E94D90366E4AE
:102D000070E080E090E00E94DF0463E873E083ED10
:102D100094E00E94D90366E470E080E090E00E94B5
:102D2000DF04A0904C01B0904D01C0904E01D090B6
:102D30004F01E0905001F09051010091520110912B
:102D40005301812C912C20E83BE346EE56E760E0EE
:102D500070E080E090E00E94C90E8091E9039091BC
:102D6000EA03029739F560E080E00E94541A6BE8AC
:102D700073E08FE396E00E94D90361E080E00E9457
:102D8000541A69EB72E08FE396E00E94D9036091D8
:102D90003C0170913D0180913E0190913F010E9464
:102DA000841A67E772E08FE396E00E94D90380E21D
:102DB0000E9430198091E9039091EA03039739F555
:102DC00060E080E00E94541A6CE973E08FE396E0C3
:102DD0000E94D90361E080E00E94541A69EB72E01E
:102DE0008FE396E00E94D90360917C0570917D0588
:102DF00080917E0590917F050E94841A69EB72E0B4
:102E00008FE396E00E94D90380E20E9430198091FE
:102E1000E9039091EA03049739F560E080E00E94AD
:102E2000541A6DEA73E08FE396E00E94D90361E0E3
:102E300080E00E94541A69EB72E08FE396E00E94F2
:102E4000D903609138017091390180913A019091D4
:102E50003B010E94841A69EB72E08FE396E00E94C6
:102E6000D90380E20E9430198091E9039091EA032E
:102E700005970CF49DC01092EA031092E90310929A
:102E80005C066091520670915306809154069091B1
:102E900055061CA21BA21EA21DA218A61FA22AE054
:102EA000AE014F5F5F4F0E94F82ABE016F5F7F4FF8
:102EB000CE0183960E9428038FA198A50B9730F529
:102EC0001AA619A61CA61BA61EA61DA64AE0BE0190
:102ED0006F5F7F4F80E090E00E94ED2ABE016F5F40
:102EE0007F4FCE0189960E942803BE016D5D7F4F02
:102EF000CE0189960E94F402BC01CE0183960E9405
:102F00003F03CE0189960E945603D6CF6BEB71E04A
:102F1000CE0101960E945B03BE016D5D7F4FCE0125
:102F200001960E94F4020E941E19BC01CE018396F4
:102F30000E943F03CE0101960E945603BE016D5DC3
:102F40007F4F83ED94E00E94B60360E570E080E07F
:102F500090E00E94DF046EEB73E0CE0101960E94C8
:102F60005B0366EB75E0CE0101960E94F4020E94BD
:102F70001E19BC0186EB95E00E943F03CE0101962D
:102F80000E94560366EB75E083ED94E00E94B60361
:102F900060E570E080E090E00E94DF046BEA72E0A0
:102FA00086EB95E00E942803CE0183960E9456038B
:102FB000AE960FB6F894DEBF0FBECDBFDF91CF91B6
:102FC0001F910F91FF90EF90DF90CF90BF90AF9047
:102FD0009F908F9008951F920F920FB60F92112419
:102FE0002F933F934F935F936F937F938F939F9311
:102FF000AF93BF93CF93DF93EF93FF93809100063E
:103000000E943304EC018091FF050E943304CC0F31
:10301000DD1F8C2BE091FE05EF7094E0E99FF0013D
:103020001124E80FF11DE956FE4F80818093FE05C3
:103030008073803119F48FEF9FEF04C0803221F448
:1030400081E090E00E94E513FF91EF91DF91CF9135
:10305000BF91AF919F918F917F916F915F914F91B0
:103060003F912F910F900FBE0F901F9018950F93C7
:103070001F93CF93DF938EE00E94C8048EE00E94DE
:10308000C804EC016AE070E080E090E00E94DF0498
:103090008EE00E94C8048EE00E94C804AC01990F23
:1030A000660B770BCE010D2E000CAA0BBB0B8A0111
:1030B0009B010D5F1F4F2F4F3F4F081719072A071E
:1030C0003B076CF04350510961097109841795075A
:1030D000A607B70724F0D0934D06C0934C06C091C5
:1030E0004C06D0914D06C53883E0D80774F0809126
:1030F0005B06811105C010924B061092580674C0F1
:10310000813031F510924B066FC0CF31D10504F5F7
:1031100080914B0681111CC0C0915B06C1110AC091
:1031200061E084E00E945C0481E080935B06809310
:10313000E80381C0C13009F057C060E084E00E941C
:103140005C0410925B061092E803C0934B064CC0DF
:10315000CE018197C99780F480914B0681110AC0F6
:103160006DEF71E088EC95E00E945C02882309F421
:1031700044C002C08130C1F1CE018B559109C49782
:1031800078F480914B06811109C063E472E088EC09
:1031900095E00E945C02882399F102C0813021F100
:1031A000CE01805991098D9778F480914B06811159
:1031B00009C06EE072E08AEA95E00E945C02882312
:1031C00051F102C0813081F0CE5BD109AB9760F440
:1031D00080914B06811108C062E473E08AEA95E0B1
:1031E0000E945C028823D1F060E070E0CB01DF91A7
:1031F000CF911F910F910C94DF0463EC73E002C038
:1032000069EC73E083ED94E00E94D90360EA70E01A
:1032100080E090E00DC06FEC73E002C063ED73E0FE
:1032200083ED94E00E94D90364EB70E080E090E0CD
:103230000E94DF0481E080934B06D6CFCF93DF93CB
:10324000EC0141E050E061E873E00E947B028111F3
:1032500003C0CE010E94E202CE01DF91CF9108951A
:10326000E0913F06F09140060190F081E02D682F3B
:103270008FE396E009948F929F92AF92BF920F9343
:103280001F93CF93DF93CDB7DEB7A1970FB6F89416
:10329000DEBF0FBECDBF19A2423008F44AE08E0156
:1032A0000F5D1F4F842E912CA12CB12CA5019401F0
:1032B0000E94362EE62FB901CA0101501109EA30E9
:1032C00014F4E05D01C0E95CD801EC93232B242BBE
:1032D000252B61F7B8018FE396E00E94C403A19605
:1032E0000FB6F894DEBF0FBECDBFDF91CF911F9117
:1032F0000F91BF90AF909F908F9008954F925F92E3
:103300006F927F928F929F92AF92BF92CF92DF92F5
:10331000EF92FF926B017C01B42E9B01AC010E94E5
:103320000D2E882319F067ED73E027C026013701C1
:10333000E89477F82FEF3FEF4FE75FE7C301B20163
:103340000E940D2E81110DC02FEF3FEF4FE75FE779
:10335000C301B2010E94682B18161CF46BED73E0D8
:103360000CC02FEF3FEF4FE75FE4C701B6010E94AB
:10337000082E181694F46FED73E08FE396E0FF903B
:10338000EF90DF90CF90BF90AF909F908F907F9005
:103390006F905F904F900C94C4032FEF3FEF4FE777
:1033A0005FECC701B6010E94682B87FDE4CF20E0E7
:1033B00030E0A901C701B6010E94682B87FF09C050
:1033C0008DE20E9430194C01F7FAF094F7F8F0946E
:1033D00002C0812C912CA12C60E070E080E09FE382
:1033E000AB1441F020E030E040E251E40E94602D57
:1033F000A394F6CF9B01AC01C701B6010E94F42C47
:103400002B013C010E94D92D6B017C010E946D2B88
:103410009B01AC01C301B2010E94F32C2B013C01C2
:103420004AE0C701B6010E943B197C01E80CF91C77
:10343000BB2029F08EE20E943019E80EF91EDB2C29
:10344000DD2021F120E030E040E251E4C301B2018F
:103450000E94CE2B2B013C010E94D92D4B01A12CA7
:10346000B12C4AE0C501B4010E943B19E80EF91ED7
:10347000C501B4010E946D2B9B01AC01C301B201D7
:103480000E94F32C2B013C01DA94DACFC701FF90A4
:10349000EF90DF90CF90BF90AF909F908F907F90F4
:1034A0006F905F904F900895CF93DF93CDB7DEB7C5
:1034B00028970FB6F894DEBF0FBECDBF28E0E3EB30
:1034C000F1E0DE01119601900D922A95E1F720912D
:1034D0004806261710F46FEF620FFE013196E60FD3
:1034E000F11DE60FF11D9081682F690F606840E0C3
:1034F0008FE396E028960FB6F894DEBF0FBECDBFDF
:10350000DF91CF910C948F05CF92DF92EF92FF92D3
:10351000CF93DF9397FF19C06B017C018DE20E946E
:103520003019EC0166277727CB016C197D098E09CC
:103530009F094AE00E943B198C0F9D1FDF91CF919C
:10354000FF90EF90DF90CF9008954AE0DF91CF9108
:10355000FF90EF90DF90CF900C943B19CF93DF93C7
:1035600000D0CDB7DEB789831A8241E050E0BE01BA
:103570006F5F7F4F82EF95E00E947B020F900F906C
:10358000DF91CF910895009769F0FC010190002030
:10359000E9F73197AF01481B590BBC0180E895E072
:1035A0000C947B0280E00895CF93DF93CDB7DEB714
:1035B000E2970FB6F894DEBF0FBECDBF789484B506
:1035C000826084BD84B5816084BD85B5826085BD1F
:1035D00085B5816085BD80916E00816080936E00AD
:1035E000109281008091810082608093810080919F
:1035F0008100816080938100809180008160809350
:1036000080008091B10084608093B1008091B0000F
:1036100081608093B00080917A00846080937A000A
:1036200080917A00826080937A0080917A00816034
:1036300080937A0080917A00806880937A0010925B
:10364000C10010926704109266041092B0041092A8
:10365000D2040E943C0710924406809148068230B2
:1036600018F098E09093440690914906992339F018
:10367000813029F48091440684608093440662E39B
:1036800070E080E090E00E94DF0460914A068FE3E2
:1036900096E00E94630568EE73E080E090E00E948F
:1036A000DF0460E38FE396E00E9476050BE416E406
:1036B000C8010197F1F760E38FE396E00E94760579
:1036C000C8010197F1F760E38FE396E00E94760569
:1036D00083E592E00197F1F760E28FE396E00E94C4
:1036E000760560914406606240E08FE396E00E94B8
:1036F0008F0584E08093450640E06CE08FE396E020
:103700000E948F0540E061E08FE396E00E948F0504
:103710000BE31FE1C8010197F1F782E080934606B1
:1037200040E066E08FE396E00E948F0540E062E0B3
:103730008FE396E00E948F05C8010197F1F788E0BA
:1037400080934A0660E08FE396E00E94630580E084
:1037500090E00E948C2C8093F203873F29F481E152
:103760000E943304892BA1F567EF69831A8280E0F8
:1037700090E06FA70E948C2C67EF681721F080E023
:1037800090E00E94942C6A8181E090E06FA70E94F3
:103790008C2C6FA5681721F081E090E00E94942C9A
:1037A00060E471E08AE090E00E94B1136CE371E0A4
:1037B00084E190E00E94B1136CE775E08EE190E047
:1037C0000E94B11368E371E088E290E00E94B113B7
:1037D00068E371E088E290E00E948B13FC01808135
:1037E0009181A281B3818115914EA105B105D1F5D9
:1037F000E091E304F091E40482E08083E091E3044B
:10380000F091E4041082E091DF04F091E004108272
:10381000E091E104F091E20480E180831092EB04F6
:10382000E091E704F091E80486E08083E091E5040C
:10383000F091E604808180618083E091E504F0915D
:10384000E604808188608083E091E504F091E604DD
:10385000808180688083E091E504F091E6048081B6
:103860008F7D808368E371E088E290E00E948B1393
:10387000FC0180819181A281B3818115924CA1408C
:10388000B105A9F5E091E304F091E40482E08083BE
:10389000E091DF04F091E0041082E091E104F09106
:1038A000E20480E180831092EB04E091E704F09160
:1038B000E80486E08083E091E504F091E6048081ED
:1038C00080618083E091E504F091E6048081886066
:1038D0008083E091E504F091E60480818068808334
:1038E000E091E504F091E60480818F7D808361E0C2
:1038F00084E00E948C0460E085E00E948C0461E01A
:1039000086E00E948C0461E087E00E948C0461E004
:1039100088E00E948C0461E089E00E948C0461E0F0
:103920008AE00E948C0461E08BE00E948C0461E0DC
:103930008CE00E948C0461E08DE00E948C0460E0C9
:1039400080E10E948C0460E081E10E948C0462E0CE
:1039500080E10E948C0462E085E00E948C0462E0B9
:1039600081E10E948C0480916800846080936800EB
:1039700080916D008C6080936D00789460E471E0BC
:103980008AE090E00E948B13FC0180819181A281EA
:10399000B3818093400190934101A0934201B09381
:1039A00043016CE371E084E190E00E948B13FC0121
:1039B00080819181A281B38180933C0190933D01EC
:1039C000A0933E01B0933F016CE775E08EE190E07B
:1039D0000E948B13DC016D917D918D919C91609380
:1039E0007C0570937D0580937E0590937F0524E68A
:1039F00030E040E050E00E94D62E20934C013093FE
:103A00004D0140934E0150934F01609350017093CC
:103A10005101809352019093530180914001909104
:103A20004101A0914201B0914301809335069093EA
:103A30003606A0933706B0933806C0903C01D0906C
:103A40003D01E0903E01F0903F011092670410921A
:103A500066041092B0041092D2040E943C0762E9FE
:103A600087EB0E946A0BC114D104E104F10409F44C
:103A70004EC08FE00E94830B682F6F73B1E8CB16A6
:103A8000B3ECDB06B9ECEB06B1E0FB0648F4C09200
:103A90003B06D0923C06E0923D06F0923E0634C0D2
:103AA000D701C6018158934CA94CB1408038934C42
:103AB000A94CB14070F4F694E794D794C794C0929F
:103AC0003B06D0923C06E0923D06F0923E066064D2
:103AD0001BC0D701C60181509748A349B340811547
:103AE0009A45A246B24080F412E0F694E794D79447
:103AF000C7941A95D1F7C0923B06D0923C06E0924B
:103B00003D06F0923E0660688FE00E946A0B60E816
:103B100080E10E946A0B60E881E10E946A0B60E824
:103B200082E10E946A0B6CE080E10E946A0B6CE00B
:103B300081E10E946A0B6CE082E10E946A0B60E204
:103B400081EB0E946A0B60E881EB0E946A0B209176
:103B50004C0130914D0140914E0150914F016091C7
:103B6000500170915101809152019091530100E0F8
:103B700010E00E94DE0CA0904C01B0904D01C0906E
:103B80004E01D0904F01E0905001F0905101009112
:103B90005201109153018091480190914901A091E7
:103BA0004A01B0914B0188529342A109B109BC016D
:103BB000CD01B2E0660F771F881F991FBA95D1F724
:103BC00024E630E040E050E00E94D62E812C912C7B
:103BD0000E94C90E80E10E94830B8C7F682F626077
:103BE00080E10E946A0B60E371E081E00E943B0B80
:103BF00068E271E082E00E943B0B60E271E083E0EA
:103C00000E943B0B68E171E084E00E943B0B60E1A5
:103C100071E085E00E943B0B68E071E086E00E9465
:103C20003B0B60E071E087E00E943B0B8090EE036D
:103C30009090EF03A090F003B090F10381149104F1
:103C4000A104B10409F492C0C0904401D090450190
:103C5000E0904601F09047016091F4037091F50304
:103C60008091F6039091F703A70196010E94582EC8
:103C7000280D391D4A1D5B1DC701B6010E94122E79
:103C80006093F4037093F5038093F6039093F70326
:103C90001AA619A61CA61BA61EA61DA62AE0AE01E2
:103CA0004F5F5F4F0E94F82ABE016F5F7F4FCE01CA
:103CB00089960E9428038DA59EA50B9730F51CA21E
:103CC0001BA21EA21DA218A61FA24AE0BE016F5F82
:103CD0007F4F80E090E00E94ED2ABE016F5F7F4F32
:103CE000CE0183960E942803BE01675D7F4FCE01FF
:103CF00083960E94F402BC01CE0189960E943F0384
:103D0000CE0183960E945603D6CF6BEB71E0CE01B5
:103D100001960E945B03BE01675D7F4FCE01019655
:103D20000E94F4020E941E19BC01CE0189960E94D5
:103D30003F03CE0101960E945603BE01675D7F4F8F
:103D400083ED94E00E94B60360E570E080E090E0CF
:103D50000E94DF041092EE031092EF031092F00322
:103D60001092F103CE0189960E9456030E943718E3
:103D70006EEB71E083ED94E00E94D90383ED94E053
:103D80000E94780166E470E080E090E00E94DF0429
:103D900083ED94E00E94FA00892B09F045C060E0B1
:103DA0008DE00E945C040E946615809118048F5F6C
:103DB000809318048091F3038F5F8093F3038091C5
:103DC000E9039091EA03892B19F00E942B16CECFBC
:103DD00060E080E00E94541A62EC71E08FE396E0AC
:103DE0000E94D90380911804863061F461E080E07C
:103DF0000E94541A63ED71E08FE396E00E94D903AC
:103E0000109218048091F3038C3009F0AFCF61E079
:103E100080E00E94541A6FE273E08FE396E00E9404
:103E2000D9031092F303A2CF61E08DE00E945C04FD
:103E300083ED94E00E94FA001816190644F583ED0C
:103E400094E00E94D80080930004893439F0809176
:103E5000FF038823E1F01092FF0319C089E40E9458
:103E6000AE1A01E083ED94E00E94FA0018161906DC
:103E700074F783ED94E00E94D800182F809300041B
:103E80000E94AE1A1B3371F70093FF03EBCF1CA205
:103E90001BA21EA21DA218A61FA262EF75E0CE01F2
:103EA00083960E943F032DE030E042E050E0BE01E7
:103EB0006D5D7F4FCE0101960E947003BE016F5F62
:103EC0007F4F84ED95E00E94A902CE0101960E94E9
:103ED000560384ED95E00E9451026093480170936F
:103EE000490180934A0190934B016093F4037093CE
:103EF000F5038093F6039093F7032EE130E04DE154
:103F000050E0BE016D5D7F4FCE0101960E947003AF
:103F1000BE016F5F7F4F8EEC95E00E94A902CE013B
:103F200001960E9456038EEC95E00E94510261308A
:103F300029F4109212046FEF71E039C0623029F455
:103F40006093120464EE71E032C0633031F484E0B7
:103F50008093120467EE71E02AC0643031F485E08A
:103F6000809312046AEE71E022C0653031F486E07D
:103F7000809312046DEE71E01AC0663031F489E06E
:103F80008093120460EF71E012C0673031F483E077
:103F90008093120463EF71E00AC0693019F06093F6
:103FA000120409C087E08093120466EF71E08EEC82
:103FB00095E00E94280321E230E040E250E0BE019B
:103FC0006D5D7F4FCE0101960E947003BE016F5F51
:103FD0007F4F88EF95E00E94A902CE0101960E94D2
:103FE000560388EF95E00E945102062F6093190452
:103FF00028E130E047E150E0BE016D5D7F4FCE012A
:1040000001960E947003BE016F5F7F4F86EE95E0C0
:104010000E94A902CE0101960E94560386EE95E009
:104020000E9451026093110429E130E048E150E020
:10403000BE016D5D7F4FCE0101960E947003BE01EF
:104040006F5F7F4F80EE95E00E94A902CE0101963E
:104050000E94560380EE95E00E9451026093100486
:1040600021E130E04DE050E0BE016D5D7F4FCE01BB
:1040700001960E947003BE016F5F7F4F88EC95E050
:104080000E94A902CE0101960E94560322E130E06F
:1040900041E150E0BE016D5D7F4FCE0101960E946F
:1040A0007003BE016F5F7F4F8CEB95E00E94A90209
:1040B000CE0101960E94560327E130E042E150E034
:1040C000BE016D5D7F4FCE0101960E947003BE015F
:1040D0006F5F7F4F82EC95E00E94A902CE010196AE
:1040E0000E94560382EC95E00E94510260930C04FA
:1040F00070930D0480930E0490930F042DE130E033
:104100004CE150E0BE016D5D7F4FCE0101960E94F3
:104110007003BE016F5F7F4F8CEE95E00E94A90295
:10412000CE0101960E9456038CEE95E00E9451024A
:10413000162F6093ED036BEA72E082EF95E00E9428
:104140002803CE0183960E945603013009F07EC0F9
:10415000113009F07BC069EF71E083ED94E00E94BB
:10416000D90383ED94E00E94780168E270E080E07A
:1041700090E00E94DF0483ED94E00E94FA0018169C
:1041800019060CF057C083ED94E00E94D80080938C
:1041900000048634A9F18091FF03882309F44AC002
:1041A00062EF75E08CE895E00E943F032DE030E07F
:1041B00044E050E06CE875E0CE0101960E94700387
:1041C000BE016F5F7F4F86E895E00E94A902CE0195
:1041D00001960E94560386E895E00E945102609382
:1041E000F8037093F9038093FA039093FB036093B1
:1041F00048017093490180934A0190934B011AC082
:1042000086E40E94AE1A01E083ED94E00E94FA0079
:10421000181619060CF0BFCF83ED94E00E94D80069
:10422000182F809300040E94AE1A1B3369F7009385
:10423000FF03EACF6BEA72E08CE895E00E94280366
:104240006BEA72E082EF95E00E9428036DEF71E067
:1042500088EC95E00E945C02882329F081E090E0E0
:10426000A0E0B0E0B5C062E072E088EC95E00E94AA
:104270005C02882329F08AE090E0A0E0B0E0A8C0CA
:1042800067E072E088EC95E00E945C02882329F0E8
:1042900082E390E0A0E0B0E09BC06CE072E088ECCC
:1042A00095E00E945C02882329F084E690E0A0E07B
:1042B000B0E08EC061E172E088EC95E00E945C02A3
:1042C000882329F08AEF90E0A0E0B0E081C066E1A9
:1042D00072E088EC95E00E945C02882329F084EF6C
:1042E00091E0A0E0B0E074C06BE172E088EC95E092
:1042F0000E945C02882329F088EE93E0A0E0B0E001
:1043000067C060E272E088EC95E00E945C0288235E
:1043100029F084EC99E0A0E0B0E05AC065E272E0D8
:1043200088EC95E00E945C02882329F088E893E1FC
:10433000A0E0B0E04DC06AE272E088EC95E00E9437
:104340005C02882329F08AE698E1A0E0B0E040C052
:104350006FE272E088EC95E00E945C02882329F00D
:1043600088E293E2A0E0B0E033C064E372E088EC5E
:1043700095E00E945C02882329F080E197E2A0E0AA
:10438000B0E026C069E372E088EC95E00E945C0230
:10439000882329F084ED90E3A0E0B0E019C06EE33B
:1043A00072E088EC95E00E945C02882329F088E99D
:1043B0009AE3A0E0B0E00CC063E472E088EC95E022
:1043C0000E945C02882361F080E29EE4A0E0B0E0FD
:1043D0008093440190934501A0934601B093470117
:1043E00060E070E0CB010E94DF040E9466150E942D
:1043F00037181091E803113091F48091FE03813059
:1044000071F068E472E083ED94E00E94D90368E201
:1044100070E080E090E00E94DF041093FE03809142
:10442000E803811112C08091FE03813071F46CE4C5
:1044300072E083ED94E00E94D90368E270E080E0CE
:1044400090E00E94DF041092FE038091ED03813022
:10445000B9F561E084E00E945C040091FC031091D6
:10446000FD030F5F1F4F1093FD030093FC0383E1D7
:104470000E94C804BC01990F880B990B0E946F2BF6
:104480006B017C0186E10E94C804BC01990F880B76
:10449000990B0E946F2B2B013C019B01AC01C701C2
:1044A000B6010E94082E87FD12C061E080E00E94E4
:1044B000541A60E572E08FE396E00E94D903A3C02E
:1044C0008111A1C060E084E00E945C049CC00115E1
:1044D000110521F0033011050CF495C0A7019601D8
:1044E000C301B2010E94F42C4B015C01A7019601AB
:1044F000C301B2010E94F32C9B01AC01C501B401C0
:104500000E94602D6B017C0120E030E0A9010E9437
:10451000082E181624F0F7FAF094F7F8F09420E03B
:1045200030E040EA50E4C301B2010E94CE2B20E00B
:1045300030EC4FE754E40E94602D2CE238E540EB6C
:104540005CE30E94602D9B01AC010E94CE2B20E019
:1045500030E048E452E40E94602D2B013C0120E051
:1045600030E040E050E4C701B6010E94F42C4B015A
:104570005C01A701960160E070E080E89FE30E9483
:10458000602D9B01AC01C501B4010E94F42C9B017C
:10459000AC0160E070E080E890E40E94602D9B0137
:1045A000AC01C301B2010E94CE2B4B015C0161E062
:1045B00080E00E94541A63E672E08FE396E00E9466
:1045C000D90342E0C701B6010E947E1961E088E08C
:1045D0000E94541A68E672E08FE396E00E94D903C5
:1045E00061E08BE00E94541A40E0C501B4010E94D2
:1045F0007E196CE672E08FE396E00E94D903109278
:10460000FD031092FC03809118048F5F80931804BF
:104610008A3009F08DC08091ED03813009F488C0A3
:104620001092180461E772E083ED94E00E94D903D0
:1046300083ED94E00E94780168E270E080E090E011
:104640000E94DF0483ED94E00E94FA001816190618
:104650000CF062C083ED94E00E94D80080930004C7
:104660008A3531F08091FF03882309F455C019C0C1
:104670008AE50E94AE1A01E083ED94E00E94FA0000
:10468000181619067CF783ED94E00E94D800182FC5
:10469000809300040E94AE1A1B3371F70093FF034E
:1046A000EBCF62EF75E084EA95E00E943F0325E0DE
:1046B00030E044E050E064EA75E0CE0101960E94EB
:1046C0007003BE016F5F7F4F8EE995E00E94A902E3
:1046D000CE0101960E9456038EE995E00E94510298
:1046E00060930B04611102C061E003C0613031F4DA
:1046F00060E087E00E945C0460E00BC0623011F46F
:1047000061E003C0633041F460E087E00E945C0434
:1047100061E086E00E945C046BEA72E084EA95E066
:104720000E9428036BEA72E082EF95E00E94280362
:104730008091E9039091EA03892B09F01EC260E0A1
:1047400083E00E94541A6091480170914901809160
:104750004A0190914B0120E432E44FE050E00E9486
:10476000582E2A30310558F480E22FA738AB49ABD8
:104770005AAB0E9430195AA949A938A92FA5CA01D4
:10478000B901882799274AE00E943B198EE20E94CE
:104790003019609148017091490180914A019091CE
:1047A0004B0120E432E44FE050E00E94582E28EE06
:1047B00033E040E050E00E94582E89012436310554
:1047C000A8F480E32FA738AB49AB5AAB0E9430194D
:1047D0002FA538A949A95AA90A30110538F480E350
:1047E0000E9430195AA949A938A92FA5CA01B901AF
:1047F000882799274AE00E943B198EE20E943019CF
:10480000609148017091490180914A0190914B015A
:1048100028EE33E040E050E00E94582E6B017C010E
:104820008B016436710548F480E30E9430190A3028
:10483000110518F480E30E943019C701B6018827DA
:1048400099274AE00E943B1960E08DE00E94541ACB
:1048500067E772E08FE396E00E94D9038091EB0353
:10486000813049F18091E80381110DC08091ED0301
:10487000811109C060E00E94541A6BE772E08FE377
:1048800096E00E94D9038091E803813021F0809165
:10489000ED03813081F46BEB72E08FE396E00E94D0
:1048A000D90360E080E00E94541A6FE772E08FE362
:1048B00096E00E94D9038091EB03813051F460E0CF
:1048C00080E00E94541A63E872E08FE396E00E9451
:1048D000D9038091ED0381115CC180910B0481119A
:1048E00009C061E00E94541A67E872E08FE396E025
:1048F0000E94D90380910B04813051F461E080E083
:104900000E94541A6CE872E08FE396E00E94D9038B
:1049100080910B04823051F461E080E00E94541ACF
:1049200061E972E08FE396E00E94D90380910B0465
:10493000833051F461E080E00E94541A66E972E02D
:104940008FE396E00E94D9032FB7F8948091E40397
:104950009091E503A091E603B091E7032FBF40914A
:104960000704509108046091090470910A04841BA3
:10497000950BA60BB70B853F9140A105B10508F437
:1049800008C16BE972E083ED94E00E94D90383EDE6
:1049900094E00E94780168E270E080E090E00E947C
:1049A000DF0483ED94E00E94FA00181619060CF05B
:1049B00049C083ED94E00E94D800809300048A35BA
:1049C00041F18091FF038823E9F162EF75E088E906
:1049D00095E00E943F0328E030E045E050E068E9C0
:1049E00075E0CE0101960E947003BE016F5F7F4F9C
:1049F00082E995E00E94A902CE0101960E94560329
:104A000082E995E00E9451027093060460930504C8
:104A100019C08AE50E94AE1A01E083ED94E00E947D
:104A2000FA00181619066CF683ED94E00E94D8007F
:104A3000182F809300040E94AE1A1B3371F7009365
:104A4000FF03EBCF6BEA72E088E995E00E94280350
:104A50006BEA72E082EF95E00E9428036BEA72E055
:104A600080E895E00E942803809105049091060457
:104A70008C3891050CF08FC344976CE070E00E9475
:104A8000222E161617060CF4A2C3109204041092DC
:104A90000304809103049091040489309105E4F0AB
:104AA00082EA92E00E94C31A61E08DE00E94541AEB
:104AB0006CEA72E08FE396E00E94D90360910104F2
:104AC00070910204072E000C880B990B0E94841A27
:104AD00080E20E94301933C08830910519F48EEAC3
:104AE00092E02BC08730910519F48EEB92E025C03F
:104AF0008630910519F48EEC92E01FC08530910547
:104B000019F48EED92E019C08430910519F48EEEFF
:104B100092E013C08330910519F48EEF92E00DC03E
:104B20008230910519F48EE093E007C0019719F4E3
:104B30008EE193E002C08EE293E00E94C31A61E02E
:104B400084E00E94541A60E875E08FE396E00E94CA
:104B5000B6032FB7F8948091E4039091E503A091F8
:104B6000E603B091E7032FBF8093070490930804F6
:104B7000A0930904B0930A040CC00E942B168091E4
:104B8000E9039091EA03059724F01092EA0310924A
:104B9000E9038091480190914901A0914A01B091A7
:104BA0004B01813A9648A140B10564F480EA96E849
:104BB000A1E0B0E08093480190934901A0934A019D
:104BC000B0934B018091480190914901A0914A0115
:104BD000B0914B01803C9540A94DB14084F080914B
:104BE000EC03813061F080EC95E0A9EDB1E08093B9
:104BF000480190934901A0934A01B0934B019091D1
:104C000012048091ED039530B9F48130A9F48091BC
:104C1000480190914901A0914A01B0914B01885FF0
:104C20009A42A109B1098093480190934901A09348
:104C30004A01B0934B0123C081111EC08091110421
:104C4000811105C0809110048111C6C208C0813055
:104C500009F066C080911004813009F0C1C28091D2
:104C6000480190914901A0914A01B0914B018852AD
:104C70009342A109B1094CC0813009F051C0809123
:104C8000110481114DC080911004813009F048C099
:104C90006CEA72E08CEB95E00E945C028823E1F004
:104CA000409148015091490160914A0170914B0136
:104CB00080910C0490910D04A0910E04B0910F040A
:104CC000840F951FA61FB71F809348019093490139
:104CD000A0934A01B0934B0160E473E08CEB95E044
:104CE0000E945C028823E1F0809148019091490183
:104CF000A0914A01B0914B0140910C0450910D04D8
:104D000060910E0470910F04841B950BA60BB70BDA
:104D10008093480190934901A0934A01B0934B01BD
:104D2000809117048F5F8F3019F08093170402C0B1
:104D300010921704409048015090490160904A0138
:104D400070904B018091130490911404A09115046C
:104D5000B0911604481659066A067B0609F462C12A
:104D6000A0904C01B0904D01C0904E01D0904F01E9
:104D7000E0905001F09051010091520110915301C7
:104D8000C301B201A2E0660F771F881F991FAA9581
:104D9000D1F724E630E040E050E00E94D62E812C8E
:104DA000912C0E94C90ED301C20180549244AF409D
:104DB000B10980389448AE41B105B8F461E08CE0A7
:104DC0000E945C0460E08BE00E945C0460E08AE08A
:104DD0000E945C0460E089E00E945C0460E088E07E
:104DE0000E945C0462E473E00CC1D301C201805CE8
:104DF000964CAD42B10980389448AE41B105B8F443
:104E000060E08CE00E945C0461E08BE00E945C0446
:104E100060E08AE00E945C0460E089E00E945C043B
:104E200060E088E00E945C0466E473E0EAC0D301BD
:104E3000C20180549B44AC44B109803C964CAD42C5
:104E4000B105B8F460E08CE00E945C0460E08BE0A7
:104E50000E945C0461E08AE00E945C0460E089E0FA
:104E60000E945C0460E088E00E945C0469E473E0F6
:104E7000C8C0D301C2019251AA47B1098115994016
:104E8000AD43B105B8F460E08CE00E945C0460E0E2
:104E90008BE00E945C0460E08AE00E945C0461E0B8
:104EA00089E00E945C0460E088E00E945C046CE49D
:104EB00073E0A7C0D301C2019B51A74BB109811573
:104EC0009940AD43B105B8F460E08CE00E945C0409
:104ED00060E08BE00E945C0460E08AE00E945C0479
:104EE00061E089E00E945C0460E088E00E945C046C
:104EF0006FE473E086C0D301C2019452A44FB1099C
:104F0000803C964CAD42B105B8F460E08CE00E9464
:104F10005C0460E08BE00E945C0460E08AE00E9438
:104F20005C0460E089E00E945C0461E088E00E942B
:104F30005C0462E573E065C0D301C201805C9A4EF7
:104F4000A142B140803C964CAD42B105B8F460E05E
:104F50008CE00E945C0460E08BE00E945C0460E0F6
:104F60008AE00E945C0460E089E00E945C0461E0E9
:104F700088E00E945C0465E573E043C0D301C20190
:104F80008058914BAF44B14080349B44AC44B10550
:104F9000B8F460E08CE00E945C0460E08BE00E946A
:104FA0005C0460E08AE00E945C0460E089E00E94AA
:104FB0005C0461E088E00E945C0468E573E021C065
:104FC000D301C201805C9C4FAB49B14080349D4508
:104FD000A64CB105D0F460E08CE00E945C0460E077
:104FE0008BE00E945C0460E08AE00E945C0460E068
:104FF00089E00E945C0461E088E00E945C046EE04D
:1050000072E08AEA95E00E94280360E070E0CB013C
:105010000E94DF044092130450921404609215041D
:10502000709216042091AE053091AF058091B405C1
:105030009091B5052817390739F58091AA05909107
:10504000AB056091B0057091B105009719F061153D
:105050007105B1F46115710551F0232B09F449C0B4
:10506000DB018C9190E09195819591090BC000979F
:1050700009F43FC0232BE9F1FC01808190E002C0DC
:105080000E942732892BA9F180911904811131C026
:1050900083E00E94830B682F6D7F83E00E946A0B80
:1050A000A0904C01B0904D01C0904E01D0904F01A6
:1050B000E0905001F0905101009152011091530184
:1050C000C301B201685B7E488F4F9F4F24E630E0FA
:1050D00040E050E00E94D62E88248394912C0E94B8
:1050E000C90E6AEA75E080EB95E00E943F031092DA
:1050F0001704809117048E3041F483E00E94830BE3
:10510000682F626083E00E946A0B8091EC0381301B
:1051100081F53090EB03F1E03F122BC083E00E9459
:10512000830B682F6B7F83E00E946A0BA0904C0179
:10513000B0904D01C0904E01D0904F01E0905001D1
:10514000F09051010091520110915301C301B2013D
:10515000685D7C4D8F4F9F4F24E630E040E050E08B
:105160000E94D62EE2E08E2E912C0E94C90E309223
:10517000EB038091EB0381110AC083E00E94830B53
:10518000682F646083E00E946A0B1092EC030E9417
:105190009A010C94161E29E030E030930404209309
:1051A0000304BC0166587109072E000C880B990B8B
:1051B0000E946F2B2FE832EC45EF5EE30E94CE2B6E
:1051C0000E94D22D709302046093010462CC70930C
:1051D0000404609303045DCC813009F0A1CD3FCD80
:1051E00081119ECDC0904801D0904901E0904A01C4
:1051F000F0904B0188E2C81A83E2D80AE108F1086E
:10520000C0924801D0924901E0924A01F0924B01CC
:105210006CEA72E08CEB95E00E945C02882309F452
:105220005BCD80910C0490910D04A0910E04B0917F
:105230000F04C80ED91EEA1EFB1EC0924801D09270
:105240004901E0924A01F0924B0146CDAF92BF92E4
:10525000CF92DF92EF92FF920F931F93CF93DF9342
:10526000E3EDF4E01382128288EE93E0A0E0B0E078
:1052700084839583A683B7832FE531E03183208330
:1052800025EC30E03587248724EC30E0378726870B
:1052900020EC30E0318B208B21EC30E0338B228B03
:1052A00022EC30E0358B248B26EC30E0378B268BDC
:1052B000118E128E138E148EE0E7F5E013821282A7
:1052C00084839583A683B78381E791E0918380836C
:1052D000EFE3F6E01382128283E891E0918380830A
:1052E00087E2848380E1808792E09187128688E05C
:1052F0008387E1E0F6E080AF81AF11AA12AA13AA7A
:105300001186128613861486158616861786108ACD
:10531000118A128A138A148A158A168A178A108E9D
:10532000118E128E138E148E158E168E178E10A25D
:1053300011A212A213A214A215A216A217A210A6BD
:1053400011A612A613A614A615A616A617A610AA8D
:1053500040EC5CEF6BE971E042AF53AF64AF75AF07
:10536000CEEFD5E0998383E08A8360E082E00E94FB
:105370008C0460E08A810E948C0461E089810E9433
:105380005C0461E08A810E945C0418826BEA72E02E
:1053900088EF95E00E945B036BEA72E082EF95E094
:1053A0000E945B036BEA72E08CEE95E00E945B0367
:1053B0006BEA72E086EE95E00E945B036BEA72E0B6
:1053C00080EE95E00E945B036BEA72E08AED95E067
:1053D0000E945B036BEA72E084ED95E00E945B0340
:1053E0006BEA72E08EEC95E00E945B036BEA72E080
:1053F00088EC95E00E945B036BEA72E082EC95E03A
:105400000E945B036BEA72E08CEB95E00E945B0309
:105410006BEA72E086EB95E00E945B036BEA72E058
:1054200080EB95E00E945B036BEA72E08AEA95E00C
:105430000E945B036BEA72E084EA95E00E945B03E2
:105440006BEA72E08EE995E00E945B036BEA72E022
:1054500088E995E00E945B036BEA72E082E995E0DF
:105460000E945B036BEA72E08CE895E00E945B03AC
:105470006BEA72E086E895E00E945B036BEA72E0FB
:1054800080E895E00E945B0320914C0130914D0132
:1054900040914E0150914F01609150017091510126
:1054A0008091520190915301E4E6AE2EB12CC12CB3
:1054B000D12CE12CF12C00E010E00E94432F20932E
:1054C0007C0530937D0540937E0550937F05DF91E9
:1054D000CF911F910F91FF90EF90DF90CF90BF90F1
:1054E000AF90089580E895E00E94560386E895E025
:1054F0000E9456038CE895E00E94560382E995E0ED
:105500000E94560388E995E00E9456038EE995E0D3
:105510000E94560384EA95E00E9456038AEA95E0C9
:105520000E94560380EB95E00E94560386EB95E0BF
:105530000E9456038CEB95E00E94560382EC95E0A6
:105540000E94560388EC95E00E9456038EEC95E08D
:105550000E94560384ED95E00E9456038AED95E083
:105560000E94560380EE95E00E94560386EE95E079
:105570000E9456038CEE95E00E94560382EF95E060
:105580000E94560388EF95E00C9456031F93FC018C
:1055900099278827BC01E89411911032E9F319305A
:1055A00010F01E30C8F31B3251F01D3249F46894DC
:1055B00006C00E94072B610F711D811D911D119165
:1055C00010531A30B0F33EF4909580957095619524
:1055D0007F4F8F4F9F4F1F910895BB274A3031F463
:1055E000992322F4BDE2909581959F4F0C943F2B17
:1055F000BB272A3051F4992342F4BDE2909580955F
:10560000709561957F4F8F4F9F4F0C941D2B592F95
:10561000482F372F262F660F771F881F991F660F79
:10562000771F881F991F620F731F841F951F660FB6
:10563000771F881F991F0895BB27FA01A62F6217AD
:10564000710581059105330B30FB66F0AA27660FC3
:10565000771F881F991FAA1FA21710F0A21B63951E
:105660003850A9F7A05DAA3308F0A95DA19336F7D9
:10567000B111B1931082CA010C94582BBB27FB01C6
:105680005527AA27880F991FAA1FA41710F0A41B3B
:1056900083955051B9F7A05DAA3308F0A95DA19395
:1056A000009779F7B111B1931192CB010C94582B5B
:1056B000DC01FC01672F71917723E1F7329704C079
:1056C0007C916D9370836291AE17BF07C8F3089504
:1056D0000E94AA2B08F481E00895E89409C097FB82
:1056E0003EF490958095709561957F4F8F4F9F4FB9
:1056F0009923A9F0F92F96E9BB279395F6958795FD
:1057000077956795B795F111F8CFFAF4BB0F11F4BF
:1057100060FF1BC06F5F7F4F8F4F9F4F16C0882366
:1057200011F096E911C0772321F09EE8872F762F9C
:1057300005C0662371F096E8862F70E060E02AF0DD
:105740009A95660F771F881FDAF7880F96958795C9
:1057500097F90895990F0008550FAA0BE0E8FEEF9E
:1057600016161706E807F907C0F012161306E40725
:10577000F50798F0621B730B840B950B39F40A261E
:1057800061F0232B242B252B21F408950A2609F4FC
:10579000A140A6958FEF811D811D08950E94E12BE8
:1057A0000C94522C0E94442C38F00E944B2C20F078
:1057B000952311F00C943B2C0C94412C11240C9447
:1057C000862C0E94632C70F3959FC1F3950F50E0D7
:1057D000551F629FF001729FBB27F00DB11D639FA3
:1057E000AA27F00DB11DAA1F649F6627B00DA11D49
:1057F000661F829F2227B00DA11D621F739FB00DEF
:10580000A11D621F839FA00D611D221F749F33275E
:10581000A00D611D231F849F600D211D822F762FF7
:105820006A2F11249F5750409AF0F1F088234AF0D4
:10583000EE0FFF1FBB1F661F771F881F9150504040
:10584000A9F79E3F510580F00C943B2C0C94862CBC
:105850005F3FE4F3983ED4F3869577956795B795C7
:10586000F795E7959F5FC1F7FE2B880F911D9695E1
:10587000879597F9089597F99F6780E870E060E051
:1058800008959FEF80EC089500240A9416161706D9
:1058900018060906089500240A9412161306140621
:1058A00005060895092E0394000C11F4882352F084
:1058B000BB0F40F4BF2B11F460FF04C06F5F7F4F3C
:1058C0008F4F9F4F089557FD9058440F551F59F023
:1058D0005F3F71F04795880F97FB991F61F09F3FDD
:1058E00079F087950895121613061406551FF2CF06
:1058F0004695F1DF08C0161617061806991FF1CF56
:1059000086957105610508940895E894BB2766277C
:105910007727CB0197F90895F999FECF92BD81BD04
:10592000F89A992780B50895262FF999FECF1FBAC6
:1059300092BD81BD20BD0FB6F894FA9AF99A0FBEB8
:10594000019608950E94E42CA59F900DB49F900DA0
:10595000A49F800D911D112408952F923F924F9284
:105960005F926F927F928F929F92AF92BF92CF92EF
:10597000DF92EF92FF920F931F93CF93DF93CDB7F8
:10598000DEB7CA1BDB0B0FB6F894DEBF0FBECDBF70
:1059900009942A88398848885F846E847D848C8441
:1059A0009B84AA84B984C884DF80EE80FD800C814A
:1059B0001B81AA81B981CE0FD11D0FB6F894DEBF2D
:1059C0000FBECDBFED010895A29FB001B39FC001EE
:1059D000A39F700D811D1124911DB29F700D811D1B
:1059E0001124911D08955058BB27AA270E940B2D02
:1059F0000C94522C0E94442C38F00E944B2C20F026
:105A000039F49F3F19F426F40C94412C0EF4E095E0
:105A1000E7FB0C943B2CE92F0E94632C58F3BA1738
:105A2000620773078407950720F079F4A6F50C94B4
:105A3000852C0EF4E0950B2EBA2FA02D0B01B90189
:105A400090010C01CA01A0011124FF27591B99F0F4
:105A5000593F50F4503E68F11A16F040A22F232F00
:105A6000342F4427585FF3CF469537952795A79550
:105A7000F0405395C9F77EF41F16BA0B620B730BF7
:105A8000840BBAF09150A1F0FF0FBB1F661F771F68
:105A9000881FC2F70EC0BA0F621F731F841F48F41D
:105AA000879577956795B795F7959E3F08F0B0CFA6
:105AB0009395880F08F09927EE0F9795879508958D
:105AC0000E94742D0C94522C0E944B2C58F00E9472
:105AD000442C40F029F45F3F29F00C943B2C5111E9
:105AE0000C94862C0C94412C0E94632C68F399230F
:105AF000B1F3552391F3951B550BBB27AA276217CA
:105B00007307840738F09F5F5F4F220F331F441FD6
:105B1000AA1FA9F335D00E2E3AF0E0E832D091500A
:105B20005040E695001CCAF72BD0FE2F29D0660FF7
:105B3000771F881FBB1F261737074807AB07B0E83A
:105B400009F0BB0B802DBF01FF2793585F4F3AF040
:105B50009E3F510578F00C943B2C0C94862C5F3FB3
:105B6000E4F3983ED4F3869577956795B795F795C6
:105B70009F5FC9F7880F911D9695879597F90895AE
:105B8000E1E0660F771F881FBB1F6217730784074A
:105B9000BA0720F0621B730B840BBA0BEE1F88F759
:105BA000E09508950E94D92D6894B1110C94862C2B
:105BB00008950E946B2C88F09F5798F0B92F992771
:105BC000B751B0F0E1F0660F771F881F991F1AF0E8
:105BD000BA95C9F714C0B13091F00E94852CB1E09C
:105BE00008950C94852C672F782F8827B85F39F09B
:105BF000B93FCCF3869577956795B395D9F73EF481
:105C000090958095709561957F4F8F4F9F4F089528
:105C10000E94AA2B08F48FEF08950E94AA2B880BEC
:105C2000990B0895DB018F939F930E94A22CBF9143
:105C3000AF91A29F800D911DA39F900DB29F900DDB
:105C40001124089597FB072E16F4009407D077FDD2
:105C500009D00E940E3007FC05D03EF49095819546
:105C60009F4F0895709561957F4F0895A1E21A2E78
:105C7000AA1BBB1BFD010DC0AA1FBB1FEE1FFF1FF0
:105C8000A217B307E407F50720F0A21BB30BE40B40
:105C9000F50B661F771F881F991F1A9469F7609587
:105CA0007095809590959B01AC01BD01CF01089541
:105CB000052E97FB1EF400940E946F2E57FD07D00F
:105CC0000E94362E07FC03D04EF40C946F2E509594
:105CD0004095309521953F4F4F4F5F4F08959095D8
:105CE0008095709561957F4F8F4F9F4F0895EE0F70
:105CF000FF1F0590F491E02D0994DF93CF931F933C
:105D00000F939A9DF02D219FF00D8B9DF00D8A9D94
:105D1000E02DF10D039FF00D029FE00DF11D4E9D52
:105D2000E00DF11D5E9DF00D4F9DF00D7F936F9383
:105D3000BF92AF925F934F93D5010E94E42C8B01E9
:105D4000AC01D7010E94E42CEB01E80FF91FD6014A
:105D50000E94CD2E2F913F91D6010E94E42CC60FB8
:105D6000D71FE81FF91FAF91BF910E94CD2E2F9131
:105D70003F910E94E42CC60FD71FE81FF91FD601E0
:105D80000E94E42CE60FF71F9801BE01CF011124F9
:105D90000F911F91CF91DF9108950E94E42C460F3F
:105DA000571FC81FD91F08F43196089597FB57FF56
:105DB0000C94E62E9F938F930E94E62E6E1B7F0B12
:105DC000AF91BF918A0B9B0B0895E894DF93CF931B
:105DD000FC01DB010E94E42C7F936F93E9019A019F
:105DE000AC01BF93AF933F932F93DF010E94E42C4C
:105DF00026F46C1B7D0B820B930B9E01EB01FC01C7
:105E00000E94CD2EAF91BF912F913F910E94CD2E38
:105E1000BE01CF01F9012F913F91CF91DF910895FC
:105E2000689401C0E894F92FF12B12F00C94442FE0
:105E3000A0E0B0E0EEE1FFE20C94B32C092E059453
:105E400022F40E94A02F112392F4F0E80F26FFEF16
:105E5000E094F09400951095B094C094D094A194DF
:105E6000BF0ACF0ADF0AEF0AFF0A0F0B1F0B0E94BF
:105E70004F2F07FC0E94A02FCDB7DEB7ECE00C94AB
:105E8000CF2C689401C0E8948F929F92CF93DF93B8
:105E90000E944F2FDF91CF919F908F90089588247B
:105EA0009924F401E401B0E49F93AA279A158B0486
:105EB0009C04ED05FE05CF05D007A10798F4AD2F92
:105EC000DC2FCF2FFE2FE92D982C892E982F872F8E
:105ED000762F652F542F432F322F2227B85031F7BA
:105EE000BF9127C01B2EBF91BB27220F331F441F1A
:105EF000551F661F771F881F991F881C991CEE1F4E
:105F0000FF1FCC1FDD1FAA1FBB1F8A149B04EC05BB
:105F1000FD05CE05DF05A007B10748F08A189B08EC
:105F2000EC09FD09CE09DF09A00BB10B21601A9421
:105F3000E1F62EF49401AF01BE01CD01000C0895ED
:105F400060957095809590953095409550952195E8
:105F50003F4F4F4F5F4F6F4F7F4F8F4F9F4F089572
:105F60000F93083090F0982F872F762F652F542F9E
:105F7000432F322F22270850F4CF220F331F441F04
:105F8000551F661F771F881F991F0A95B2F70F913B
:105F9000089597FB10F8169400080F93083098F0B6
:105FA0000850232F342F452F562F672F782F892FF6
:105FB000902DF4CF0594979587957795679557958C
:105FC0004795379527950A95AAF70F9108952A0DB9
:105FD0003B1D4C1D5D1D6E1D7F1D801F911F089573
:105FE0002A193B094C095D096E097F09800B910B49
:105FF00008952A153B054C055D056E057F05800754
:10600000910708950024A7FD00942A173005400544
:10601000500560057005800590050895AA1BBB1BFF
:1060200051E107C0AA1FBB1FA617B70710F0A61B98
:10603000B70B881F991F5A95A9F780959095BC01B9
:10604000CD010895CF93DF938230910510F482E063
:1060500090E0E0915F06F091600620E030E0C0E063
:10606000D0E0309711F14081518148175907C0F0B5
:106070004817590761F482819381209719F09B8317
:106080008A832BC09093600680935F0626C02115FB
:10609000310519F04217530718F49A01BE01DF01C8
:1060A000EF010280F381E02DDCCF2115310509F1EC
:1060B000281B390B2430310590F412968D919C9158
:1060C00013976115710521F0FB019383828304C04E
:1060D0009093600680935F06FD01329644C0FD01F7
:1060E000E20FF31F81939193225031092D933C933A
:1060F0003AC020915D0630915E06232B41F4209139
:1061000057013091580130935E0620935D0620912F
:106110005501309156012115310541F42DB73EB797
:106120004091590150915A01241B350BE0915D06B5
:10613000F0915E06E217F307A0F42E1B3F0B281721
:10614000390778F0AC014E5F5F4F2417350748F0F0
:106150004E0F5F1F50935E0640935D0681939193AF
:1061600002C0E0E0F0E0CF01DF91CF9108950F93FE
:106170001F93CF93DF93009709F48CC0FC013297F3
:106180001382128200915F061091600601151105BD
:1061900081F420813181820F931F20915D0630911F
:1061A0005E062817390779F5F0935E06E0935D06E1
:1061B00071C0D80140E050E0AE17BF0750F412960E
:1061C0002D913C911397AD012115310509F1D901AC
:1061D000F3CF9D01DA013383228360817181860FC1
:1061E000971F8217930769F4EC0128813981260FE4
:1061F000371F2E5F3F4F318320838A819B8193839A
:106200008283452B29F4F0936006E0935F0642C039
:106210001396FC93EE931297ED01499159919E01CB
:10622000240F351FE217F30771F480819181840FE9
:10623000951F029611969C938E938281938113965B
:106240009C938E931297E0E0F0E0D80112968D9126
:106250009C911397009719F0F8018C01F6CF8D915E
:106260009C9198012E5F3F4F820F931F20915D06F6
:1062700030915E062817390769F4309729F4109297
:10628000600610925F0602C01382128210935E06AF
:1062900000935D06DF91CF911F910F910895A0E0CB
:1062A000B0E0E5E5F1E30C94B12CEC01009721F4AA
:1062B000CB010E942230B8C0FC01E60FF71F9C0101
:1062C00022503109E217F30708F4ACC0D9010D914F
:1062D0001C91119706171707B0F00530110508F447
:1062E0009FC0C80104978617970708F499C0025009
:1062F0001109061B170B019311936D937C93CF012A
:106300000E94B7308DC05B01A01AB10A4C01800E0B
:10631000911EA0915F06B091600640E050E0E12C34
:10632000F12C109709F44AC0A815B905D1F56D9064
:106330007C901197630182E0C80ED11CCA14DB0463
:1063400080F1A3014A195B096A0182E0C80ED11CE1
:106350001296BC9012971396AC91B5E0CB16D1046F
:1063600040F0B282A38351834083D9016D937C9323
:106370000AC00E5F1F4FC301800F911FF901918367
:106380008083EB2DFA2FE114F10431F0D70113963D
:10639000FC93EE93129744C0F0936006E0935F067F
:1063A0003FC08D919C9111974817590708F4AC0193
:1063B0007D0112960D90BC91A02DB3CF80915D060A
:1063C00090915E0688159905E1F446175707C8F4C1
:1063D0008091550190915601009741F48DB79EB779
:1063E0004091590150915A01841B950BE817F90708
:1063F000C8F4F0935E06E0935D06F9017183608353
:106400000FC0CB010E9422307C01009759F0A801F7
:10641000BE010E941E32CE010E94B730C70104C0E7
:10642000CE0102C080E090E0CDB7DEB7EEE00C9484
:10643000CD2C81E090E0F8940C943732FB01DC0124
:1064400002C001900D9241505040D8F70895FB01D1
:10645000DC018D91019080190110D9F3990B0895F9
:10646000FB01DC0101900D920020E1F7089510E09E
:10647000C2E7D0E004C0FE010E94772E2196C33708
:08648000D107C9F7F894FFCF22
:106488001F1115111D1D111F1F1115111515111F94
:106498001F111D1D1D1D1D1F1F1117111515111F62
:1064A8001F1117111D1D111F1F1515111D1D1D1F52
:1064B8001F111D111D1D111F00E10000C0FC9B01D3
:1064C800E86E030064000000A03B4C0000046BF47D
:1064D8001400000001000061068000000000003187
:1064E800019E00C9007801FA00D800EC0000000005
:1064F800005C130C075913FC0120020C02FD01007B
:10650800000000B0059E0059135813000000002831
:10651800029E0059135813000204000300011003DF
:106528000200000302010006000400060500200620
:10653800050400000040001400540046410049468C
:106548003B0020204E6F20636F6E6E656374696F29
:106558006E200020202020506F776572534452200F
:106568002020200030320030340030350030360032
:1065780030390030330030370046423B003030308D
:106588003000303030310031303030003030313090
:1065980000313030310031303130003030313100AD
:1065A800313031310031313030003031303000306D
:1065B800313031003131303100313131300030315A
:1065C800313000303131310054583B0052583B00D3
:1065D800535752202020202020503D305720202083
:1065E8002020005357523D0020503D0057202020C6
:1065F800005A5A50413B0020487A00525820005413
:1066080058200056464F004F666620004C6F772092
:10661800004D6564200048696768005A5A534D3038
:106628003B00FFFFFFFFFFFFFFFF07002B00FFFFFF
:10663800FFFFFFFFFF062020202020202000FFFF73
:10664800FFFFFFFF05202020202020202000FFFF43
:10665800FFFFFF0420202020202020202000FFFF13
:10666800FFFF032020202020202020202000FFFFE3
:10667800FF02202020202020202020202000FFFFB3
:106688000120202020202020202020202000FFFF83
:106698002020202020202020202020202000FF2033
:1066A8002020202020202020202020202000202002
:1066B80020202020202020202020202020202000F2
:1066C8002D0031363000383000343000333000329D
:1066D80030003137003135003132002031392E3960
:1066E80034382E303030204D487A2000436F7252B3
:1066F8006566200046413030303034393936303024
:10670800303B005A5A4D4430323B00436F72724658
:106718005245512E2051554152545A0020436F7210
:10672800722E504C4C5F46495845442000434F4D0B
:1067380020504F52542052532D32333220005A5A8F
:106748004D44005A5A53443B005A5A53553B004251
:10675800553B0042443B006E616E00696E66006FF7
:046768007666000051
:00000001FF
